:1000000000400020A9500000E9500000EB50000023
:1000100000000000000000000000000000000000E0
:10002000000000000000000000000000ED50000093
:100030000000000000000000EF500000F150000040
:10004000F35000005D39000025550000F35000001A
:10005000F350000000000000F3500000F3500000D7
:10006000F3500000F5570000F3500000F35000007B
:10007000F3500000F3500000F3500000F350000074
:10008000F35000008D590000F3500000F3500000C1
:10009000F3500000F3500000F3500000F350000054
:1000A000F3500000F35000000000000000000000CA
:1000B0000000000000000000000000000000000040
:1000C00010B5064C2378002B07D1054B002B02D02E
:1000D000044800E000BF0123237010BD440200204B
:1000E0000000000048B70000044B10B5002B03D0FF
:1000F0000349044800E000BF10BDC04600000000F6
:100100004802002048B70000164B002B00D1144BCA
:100110009D46402292029A1A924600218B460F4633
:100120001348144A121A08F072FD0F4B002B00D02E
:1001300098470E4B002B00D0984700200021040068
:100140000D000D48002802D00C4800E000BF08F068
:100150001DFD2000290005F003FA08F0F1FCC0465F
:100160000000080000400020000000000000000027
:1001700044020020C0250020000000000000000014
:1001800002000120104004D1042A01D9106800099E
:1001900070470020FCE710B50400FFF7F1FF0028CE
:1001A00009D001388000031D22181279002A02D0DC
:1001B00001309842F8D110BD0122096810B51142F2
:1001C00001D0002903DA102000F084F910BD491095
:1001D000062002F05DF8F9E7096810B5CB0701D5F4
:1001E000002903DA102000F075F910BD4910033121
:1001F00089100022052002F04BF8F6E770B50D6873
:10020000AB0729D1042D27D90F232A684E68134044
:10021000062B0BD12800FFF7B3FF0123984201DA28
:1002200000200AE09A00AE500133F7E7052B13D106
:10023000F30703D4132000F04DF970BD7610FF2EA4
:10024000F8D82800FFF79CFF2C1D80002018A04242
:10025000E6D926700134FAE70B2000F03BF9DFE71E
:1002600070B50C681120E30712D54D68AB072BD190
:10027000042D29D90F262B6864101E40062E0DD19F
:10028000002C04DD2800FFF77BFFA04203DA1220D8
:1002900000F020F901E0A400605970BD331F012B6C
:1002A00012D82800FFF76CFF8000042E02D128002E
:1002B000FFF771FF002CEADDA042E8DB01202C19DA
:1002C000E3785B001843E8E70B20E1E7F8B501238A
:1002D0000D6811201D4214D003244E6834402CD1E7
:1002E000042E2AD90F2332686D108F681340062B15
:1002F0000ED1002D04DD3000FFF742FFA84203DAE3
:10030000122000F0E7F802E0AD00AF512000F8BD88
:10031000052B12D1002DF3DD3000FFF731FF8000F7
:10032000A842EDDB01231F4201D11320E9E77F1032
:10033000FF2FFAD87519EF70E8E70B20E1E708689E
:1003400010B5830717D1042815D90F23026813406D
:10035000062B03D1FFF714FF430004E0052B05D162
:10036000FFF70EFFC3000120184310BD042B02D17C
:10037000FFF711FFF0E70B2000F0ACF8F5E7000005
:1003800002000120104001D0501070470D22014B97
:100390001A70FAE78402002002000120104004D104
:1003A000042A01D91068000970470020FCE770B5E5
:1003B0000E000400FFF7F0FF05003000FFF7ECFF30
:1003C0000023854206D10434AD0004366519AC42E1
:1003D00002D30123180070BD20783278002801D1A3
:1003E000002AF6D0013401369042F0D00023F1E724
:1003F000F0B585B00393019002912D4E2D4B002A4C
:1004000002D002223270013A00251A601B68F554AE
:10041000019B9D4201DB05B0F0BD029AAB00D058B4
:10042000244B1C68C8239B0037191C1B012318424E
:1004300006D0214A43102100380008F0B5FF09E03A
:100440001E4A002802D004281BD11D4A2100380072
:1004500008F0AAFF300009F00BF8164A039B106061
:10046000002B0CD0019B013BAB4208DD154B9842A1
:1004700005D8431C1360202232540022F254013567
:10048000C6E7042810D90F2302681340042B04D1B7
:1004900001F03AFF0C4A0300CDE7062B05D1FFF728
:1004A0007BFF0A4A0300C6E70123094AC3E7C046A7
:1004B00085020020A8050020FDA30000D0A30000B5
:1004C000D6A300001F030000DBAF0000DBA3000089
:1004D000ECA30000014B187000207047840200203C
:1004E00070B501F0E9FC094C0100251D1F22280010
:1004F00008F0C5FF280008F0BBFF04230430800883
:10050000000118432060200070BDC046600200203A
:10051000C368F0B59D00836889B05D190300183386
:1005200006930369069A9F00069B0390DF194369AF
:1005300001939B00D3180293CD4B1B78002B26D13F
:100540007F222B68CB491C1213409B005B5804355B
:1005500001929F46039B587803F098FE0023039A6C
:10056000137027E0C24B1B78002B10D12B68019A27
:100570001C121340BF4A9B009B580435E9E7069BB9
:100580003A1DD11ABA4BD82928DD1A221A70039BBA
:10059000B74C9B6821780193EA1A039B92109B78D1
:1005A00012021A43039B587803F078FE0023039A43
:1005B00023701370039B069A9B680193ED1A039BAB
:1005C000AD10DD60069BFE1A039BB6101E61029BF8
:1005D0009B1A039A9B10536109B0F0BD1B783C60D5
:1005E000002B01D01700D2E72B6801991C120B4099
:1005F000A0499B005B5817000435AAE7069B3A1DEB
:10060000D11A9B4BD82902DD1A221A70BFE728683D
:100610001B78291D3860002B02D017000D00B6E7AB
:100620006B6801991C120B4092499B005B581700A4
:1006300008358EE7069B3A1DD11A8D4BD82902DD6D
:100640001A221A70A3E7A4001B782C193C60002B17
:1006500001D017009BE72B6801991C120B408549BC
:100660009B005B581700043573E7069B3A1DD11AAF
:100670007F4BD82902DD1A221A7088E77E49A40030
:1006800061581B783960002B01D017007FE72B6879
:1006900001991C120B4077499B005B5817000435E9
:1006A00057E7043F744B3A68A400E250704B1B7844
:1006B000002B00D06BE72B68019A1C1213406D4A87
:1006C0009B009B58043544E76B4BA400E058FFF7B0
:1006D00057FE043F06003868FFF752FE3618012027
:1006E000654B76000643E650614B1B78002B00D02B
:1006F0004DE72B68019A1C1213405E4A9B009B58E1
:10070000043526E7069B3A1DD11A594BD82902DD3C
:100710001A221A703BE70698029C0121A04202D2DD
:1007200021000C3909681B783960002B01D01700B3
:100730002DE72B6801991C120B404E499B005B581A
:100740001700043505E7069B3A1DD11A484BD829F6
:1007500002DD1A221A701AE70699029881420FD216
:1007600003000C3B1B6845495B106418E41AA400A5
:1007700023583B603E4B1B78002B05D0170006E743
:10078000182119700023F4E72B6801991C120B4003
:1007900038499B005B5817000435DAE6069B029A3D
:1007A000934219D213000C3B1B68344A043FA4182F
:1007B0005B10E31A029A39689B0099502C4B1B7806
:1007C000002B00D0E3E62B68019A1C121340294A43
:1007D0009B009B580435BCE61822254B1A70EDE7A8
:1007E000069B029A93422DD2244B3E1FE31814001D
:1007F0000C3C04932368049A5B10D31A029A9B0062
:100800009858FFF7BDFD07903068FFF7B9FD2468E1
:10081000049B64101C1B079BA4001F1801207F0071
:10082000029B0743E7503700114B1B78002B00D089
:10083000ADE62B68019A1C1213400E4A9B009B5890
:10084000043586E618220A4B1A70EDE7069B3A1D1E
:10085000D11A074BD82902DD1A221A7097E602999D
:10086000A40061581B783960002B09D017008EE670
:1008700084020020D0A1000068230020FDFFFF3F7C
:100880002B6801991C120B40D8499B005B5817003C
:1008900004355EE6043F029B3A68A400E250D44B64
:1008A0001B78002B00D072E62B68019A1C121340B3
:1008B000CE4A9B009B5804354BE6029BA4001C19B2
:1008C0002368043F38685E10FFF75AFD3618012090
:1008D000C74B76001B7806432660002B00D056E6F7
:1008E0002B68019A1C121340C04A9B009B58043588
:1008F0002FE6069BA4003F1BBD4CBB420CD82378BF
:10090000002B00D043E62B68019A1C121340B74A13
:100910009B009B5804351CE6B64801F069FC23781F
:10092000002B00D033E62B68019A1C121340AF4A0B
:100930009B009B5804350CE6A300ED18002C00DA50
:1009400038E6AB4B1B78002B00D020E62B68019AD1
:100950001C121340A54A9B009B580435F9E5043F3F
:100960003B68042B04D1A300ED18002C00DA21E62B
:100970009F4B1B78002B00D009E62B68019A1C12B4
:1009800013409A4A9B009B580435E2E5043F3B68BC
:10099000042B06D0A200AD18002C02DA002B00D1E7
:1009A00008E6934B1B78002B00D0F0E52B68019AEA
:1009B0001C1213408D4A9B009B580435C9E53A1F11
:1009C00013685B10013B002B06DD01215B00A400D6
:1009D0000B432D191360EDE5854B17001B78002B99
:1009E00000D0D4E52B68019A1C1213407F4A9B006B
:1009F0009B580435ADE53A00069B0C32D31AD82B30
:100A000003DD1A227A4B1A70C1E5FF2361005B00F7
:100A10001940FE3BFF3B19433960039906988968EA
:100A2000241204916D1A0399AD1089782D020D439B
:100A300002999D40091A891099401D430B43BB60E0
:100A4000039B7D609C70E4B26B4BE4000292E35820
:100A5000039A9360664A1278002A03D008331D0077
:100A6000029F94E51D00019A9B680C351C121340EF
:100A70005E4A9B009B58029F6BE53B1F1C68029AD5
:100A8000069B93422FD10A20E3070ED4A30715D16A
:100A9000042C13D90F2322681340042B11D12000FA
:100AA00001F032FC08F0E4FC0630643003F0DCF8BE
:100AB00000280FD1043D069B02937BE50720042C00
:100AC000F3D02000431E9841FA234042FF331840E0
:100AD0000730EAE7039B2100587803F0F1FB00237D
:100AE000039A1370E7E7029B029A0C3B1B68039979
:100AF0005B109B00D31A0C3B1C601F1D1300083BAE
:100B00001B685A108A70D2B23B49D2005B0055581C
:100B10009B0A039A9B009560ED18029B069A043B82
:100B20001B685B109B00D3180293314B1B78002B82
:100B300000D02CE52B68019A1C1213402B4A9B0015
:100B40009B58043505E53B1F1868FFF719FCA40006
:100B500006003F1B1E2827DC00280DDC244B1B78D9
:100B6000002B00D013E52B68019A1C1213401F4A7A
:100B70009B009B580435ECE401F08CF9033E3618D9
:100B800001F088F91D4B801B9842F9D8184B1B784F
:100B9000002B00D0FBE42B68019A1C121340134A6F
:100BA0009B009B580435D4E40123039A137001F091
:100BB00071F9039B0A3886195E60FBE43B1F1868D5
:100BC000FFF7DEFBA40006003F1B002818DC084BE3
:100BD0001B78002B00D0DAE42B68019A1C1213401A
:100BE000024A9B009B580435B3E4C046D0A10000E4
:100BF0008402002000A40000701B00209F860100DA
:100C0000C64B984203DD1D22C54B1A70BFE4012379
:100C1000039A137001F03EF9FA239B005E43039B95
:100C20000A3E30185860C5E4A300FF1A00232000D4
:100C30001A003900FFF7DCFBBA4EBB4C31682000CC
:100C400003F0F6F93168200003F041FB3168200021
:100C500001F0F0FBB24B1B78002B00D097E42B681F
:100C6000019A1C121340B14A9B009B58043570E452
:100C7000AB4BA4001B783F1B002B00D087E42B68F4
:100C8000019A1C121340A94A9B009B58043560E44A
:100C9000039803F04DF8A24B1B78002B00D076E4AC
:100CA0002B68019A1C121340A04A9B009B580435E4
:100CB0004FE43B1F1868002838D1083B1868C30769
:100CC0001ED540103A0001234100083A0B4313603F
:100CD000002859DD01234200391F1A430A603A00F7
:100CE000083A12681A41101A3A000C3A116819426F
:100CF0001FD0C0189840A4001843029BE05027E082
:100D000083070FD104280DD90F2302681340062B47
:100D100002D1FFF741FBD5E7052B03D1FFF73CFBE1
:100D20008000CFE719227E4B1A7030E44010013862
:100D3000CEE78A0723D1042921D90F220E68324039
:100D4000062A15D1013080004358029AA400A3500E
:100D5000734B1B78002B01D0FFF719FC2B68019A0D
:100D60001C121340714A9B009B580435FFF7F1FB9E
:100D7000052A04D108180079A4004000BCE7192214
:100D8000674B1A70FFF703FC0435E1E7A300069AEE
:100D9000FB189B1AD82B13DC0122631E002C14DCD9
:100DA0005F4B1B78002B01D0FFF7F1FB2B68019AFA
:100DB0001C1213405D4A9B009B580435FFF7C9FB8A
:100DC0001A22574B1A70FFF7E2FB3A601C000437F7
:100DD000E3E7069A3B1D9B1A514ED82B03DD1A23DD
:100DE0003370FFF7D4FB069B029AA40093422AD2E9
:100DF0003B1F1868FFF7C4FA011E21DD029B0C3B64
:100E00001A68521082421BDB9007801A484B401828
:100E1000C018029B8000C2583B1B1A60404B3F1B0E
:100E20001B780437002B01D0FFF7B1FB2B68019A28
:100E30001C1213403D4A9B009B580435FFF789FB69
:100E400020233370EAE71823FBE7A3009C46FE1A31
:100E5000002C17DC1C22324B1A70002333606346CF
:100E6000FF1A2F4B04371B78002B01D0FFF78FFBA5
:100E70002B68019A1C1213402C4A9B009B58043586
:100E8000FFF767FB002033685A108300F1580123F5
:100E90000B4003D10D21224A1170DFE749108A422D
:100EA00000DD0A0001308442EFDC012352001343CD
:100EB000D4E7A3009C46FE1A002C17DC1C22184B1A
:100EC0001A70002333606346FF1A154B04371B78F2
:100ED000002B01D0FFF75BFB2B68019A1C1213401B
:100EE000124A9B009B580435FFF733FB0020336800
:100EF0005A108300F15801230B4003D10D21084AF9
:100F00001170DFE749108A4200DA0A00013084429A
:100F1000EFDC012352001343D4E7C04680EE3600D5
:100F200084020020A805002085020020D0A1000036
:100F3000FCFFFF3F3B00083B1868FFF721FA3B1F0F
:100F400006001868FFF71CFA0023864200DA043313
:100F5000A4003A1B17001360E34B04371B78002BE7
:100F600001D0FFF714FB2B68019A1C121340DF4AD3
:100F70009B009B580435FFF7ECFA3B00083B1868D0
:100F8000FFF7FEF93B1F06001868FFF7F9F9F30FAA
:100F9000C217B0425341A4003A1B17009B001360D4
:100FA000D14B04371B78002B01D0FFF7F0FA2B68E8
:100FB000019A1C121340CD4A9B009B580435FFF741
:100FC000C8FA3B00083B18683B1F1968A600BE1B07
:100FD0000423814202D0042802D8002333601CE09D
:100FE0000123184201D01942F7D103239C4618422D
:100FF000F3D102680C331A40042AEED16246114242
:10100000EBD10429E9D90A681340042BE5D1FFF795
:10101000CEF9431E984180003060B34BA4001B788A
:101020003F1B0437002B01D0FFF7B1FA2B68019A60
:101030001C121340AD4A9B009B580435FFF789FAF8
:101040003B00083B18683B1F1968A600BE1B002325
:10105000814202D0042802D8042333601CE001231B
:10106000184201D01942F7D103239C461842F3D10C
:1010700002680C331A40042AEED162461142EBD1C9
:101080000429E9D90A681340042BE5D1FFF78FF949
:101090004342584180003060934BA4001B783F1BB3
:1010A0000437002B01D0FFF772FA2B68019A1C124B
:1010B00013408E4A9B009B580435FFF74AFA3B00C9
:1010C000083B1868FFF75CF93B1F06001868FFF73C
:1010D00057F9F317C20F86425341A4003A1B170079
:1010E0009B001360804B04371B78002B01D0FFF767
:1010F0004EFA2B68019A1C1213407C4A9B009B58A5
:101100000435FFF726FA3B00083B1868FFF738F96B
:101110003B1F06001868FFF733F90023864200DD05
:101120000433A4003A1B170013606F4B04371B787D
:10113000002B01D0FFF72BFA2B68019A1C121340E9
:101140006A4A9B009B580435FFF703FA3B1F1B6854
:10115000A400043B5A1E93413A1B17009B001360E6
:10116000614B04371B78002B01D0FFF710FA2B6876
:10117000019A1C1213405D4A9B009B580435FFF7EF
:10118000E8F93B00083B1868FFF7FAF83B1F060038
:101190001868FFF7F5F832180120A4003B1B1F0068
:1011A000520002431A60504B04371B78002B01D0C9
:1011B000FFF7EDF92B68019A1C1213404B4A9B0074
:1011C0009B580435FFF7C5F93B00083B1868FFF74B
:1011D000D7F83B1F06001868FFF7D2F8321A012033
:1011E000A4003B1B1F00520002431A603E4B043711
:1011F0001B78002B01D0FFF7CAF92B68019A1C124B
:1012000013403A4A9B009B580435FFF7A2F93B0074
:10121000083B1868FFF7B4F83B1F06001868FFF793
:10122000AFF802000120A4003B1B1F0072435200D4
:1012300002431A602C4B04371B78002B01D0FFF7B8
:10124000A6F92B68019A1C121340284A9B009B5850
:101250000435FFF77EF93B1F1868FFF791F8061E6B
:1012600017D11F22204B1A70A4003B1B1F001E60C9
:101270001D4B04371B78002B01D0FFF788F92B6832
:10128000019A1C121340194A9B009B580435FFF722
:1012900060F93B00083B1868FFF772F8310005F071
:1012A00095FE012640000643DEE73B1F1868FFF766
:1012B00067F8061E1CD11F220B4B1A70A4003B1BA3
:1012C0001F001E60084B04371B78002B01D0FFF76E
:1012D0005EF92B68019A1C121340044A9B009B582C
:1012E0000435FFF736F9C04684020020D0A1000083
:1012F0003B00083B1868FFF743F8310005F04CFF4E
:10130000012649000E43D9E73B1F1868FFF738F85C
:10131000C217801850400122A4003B1B1F00400050
:1013200010431860F14B04371B78002B01D0FFF7F6
:101330002EF92B68019A1C121340ED4A9B009B5812
:101340000435FFF706F9A300FE1A3068012C24D1FA
:10135000FFF716F80494079007F0E2FF07990029B9
:1013600000DC012105F018FF049BA400C91801232B
:1013700049001943DD4B3F1B1B7831600437002BBC
:1013800001D0FFF704F92B68019A1C121340D84AC8
:101390009B009B580435FFF7DCF8FEF7F1FF049043
:1013A0007068FEF7EDFF049B0130C31A0793D3E783
:1013B000A300FE1A31002000049300F0DBFF049B21
:1013C0003060FF1AC94B04371B78002B01D0FFF7A0
:1013D000DEF82B68019A1C121340C54A9B009B58EB
:1013E0000435FFF7B6F83B00083B1868FEF7C8FF66
:1013F0003B1F06001868FEF7C3FF02000120A4008F
:101400003B1B1F003240520002431A60B74B0437A7
:101410001B78002B01D0FFF7BAF82B68019A1C1239
:101420001340B34A9B009B580435FFF792F83B00EA
:10143000083B1868FEF7A4FF06003B1F1868FEF77C
:101440009FFF320002430120A4003B1B1F005200FB
:1014500002431A60A54B04371B78002B01D0FFF71D
:1014600096F82B68019A1C121340A14A9B009B58C6
:101470000435FFF76EF83B00083B1868FEF780FF65
:1014800006003B1F1868FEF77BFF32004240012038
:10149000A4003B1B1F00520002431A60934B043709
:1014A0001B78002B01D0FFF772F82B68019A1C12F1
:1014B00013408F4A9B009B580435FFF74AF83B1FA7
:1014C0001868FEF75DFFC0430122A4003B1B1F000C
:1014D000400010431860854B04371B78002B01D067
:1014E000FFF755F82B68019A1C121340804A9B00A5
:1014F0009B580435FFF72DF83B00083B1868FEF7B2
:101500003FFF06003B1F1868FEF73AFF320082409B
:1015100051000122A4003B1B1F000A431A60734BB9
:1015200004371B78002B01D0FFF731F82B68019AA4
:101530001C1213406E4A9B009B580435FFF709F8B4
:101540003B00083B1868FEF71BFF06003B1F1868AE
:10155000FEF716FF3200024151000122A4003B1B9E
:101560001F000A431A60614B04371B78002B01D01F
:10157000FFF70DF82B68019A1C1213405C4A9B0080
:101580009B580435FEF7E5FF3B000C3B1868FEF75F
:10159000F7FE3B00083B06001868FEF7F1FEF11766
:1015A0000200C317300005F049FE3B1F049005916F
:1015B0001868FEF7E5FE02000498059905F0F2FDB3
:1015C00043000120A4003E1B37001843474B306006
:1015D0001B780437002B01D0FEF7D9FF2B68019A46
:1015E0001C121340424A9B009B580435FEF7B1FF82
:1015F000A300FE1A310020000493FEF7DDFD049BDA
:101600003060FF1A394B04371B78002B01D0FEF7EE
:10161000BEFF2B68019A1C121340354A9B009B5851
:101620000435FEF796FFA300FE1A31002000049354
:10163000FEF7D2FD049B3060FF1A2C4B04371B7859
:10164000002B01D0FEF7A3FF2B68019A1C12134058
:10165000274A9B009B580435FEF77BFFA300FF1A27
:1016600039002000FEF7CAFD204B1B78002B01D06B
:10167000FEF78DFF2B68019A1C1213401C4A9B0039
:101680009B580435FEF765FFA300FE1A31002000C9
:101690000493FEF7E5FD049B3060FF1A134B0437FB
:1016A0001B78002B01D0FEF772FF2B68019A1C12E9
:1016B00013400F4A9B009B580435FEF74AFFA300D6
:1016C000FF1A39002000FEF701FE084B1B78002BA3
:1016D00001D0FEF75CFF2B68019A1C121340044AEC
:1016E0009B009B580435FEF734FFC046840200205F
:1016F000D0A10000A300FE1A310020000493FEF7E1
:101700001EFE049B3060FF1AF24B04371B78002B3F
:1017100001D0FEF73CFF2B68019A1C121340EE4AE1
:101720009B009B580435FEF714FF069B3E1DF31AE1
:10173000E84CD82B03DD1A232370FEF728FF00F0B6
:10174000B3FB43000120184323783860002B02D0FC
:101750003700FEF71CFF2B68019A1C121340DE4A6B
:101760009B009B5837000435FEF7F3FE069B3E1D99
:10177000F31AD84CD82B03DD1A232370FEF707FF8A
:1017800000F088FBD54B4000184001231843237814
:101790003860002B02D03700FEF7F9FE2B68019A63
:1017A0001C121340CC4A9B009B5837000435FEF7AF
:1017B000D0FE0123A600BE1B20001A003100FEF758
:1017C00017FEC74C2068643002F04EFA002802D1A0
:1017D000043DFEF7EFFE039B21685A78C14802F0F2
:1017E00084FD0123039A3700137000F053FBBE4BB6
:1017F00022681B68063253431818039B5860FEF793
:10180000D9FEA600BE1B2000012300223100FEF7F6
:10181000EFFDB34C2068643002F026FA0028D7D0E0
:10182000B04802F05DFBDCE7A4003E1BFEF758FE6B
:101830003700A84B30601B780437002B01D0FEF72F
:10184000A6FE2B68019A1C121340A34A9B009B58CA
:101850000435FEF77EFEA4003E1B300000F053FB73
:1018600037009C4B30601B780437002B01D0FEF70B
:101870008EFE2B68019A1C121340974A9B009B58BE
:101880000435FEF766FEA4003E1B300000F03DFB71
:101890003700904B30601B780437002B01D0FEF7E7
:1018A00076FE2B68019A1C1213408B4A9B009B58B2
:1018B0000435FEF74EFEA300FE1A3100200004930B
:1018C00000F026FB049B3060FF1A824B04371B7824
:1018D000002B01D0FEF75BFE2B68019A1C1213400F
:1018E0007D4A9B009B580435FEF733FEA4003F1B46
:1018F000380000F03FFB774B1B78002B01D0FEF740
:1019000046FE2B68019A1C121340734A9B009B5899
:101910000435FEF71EFEA300FE1A310020000493DA
:1019200000F050FB049B3060FF1A6A4B04371B78B1
:10193000002B01D0FEF72BFE2B68019A1C121340DE
:10194000654A9B009B580435FEF703FEA4003F1B2D
:10195000380000F079FB5F4B1B78002B01D0FEF7BD
:1019600016FE2B68019A1C1213405B4A9B009B5881
:101970000435FEF7EEFD0121200000F04DFB554B34
:101980001B78002B01D0FEF702FE2B68019A1C1277
:101990001340514A9B009B580435FEF7DAFD0021A5
:1019A000200000F039FB4B4B1B78002B01D0FEF7D9
:1019B000EEFD2B68019A1C121340474A9B009B586E
:1019C0000435FEF7C6FDA4003E1B300000F05EFBB0
:1019D0003700404B30601B780437002B01D0FEF7F6
:1019E000D6FD2B68019A1C1213403B4A9B009B5862
:1019F0000435FEF7AEFDA4003E1B300000F05AFB9C
:101A00003700344B30601B780437002B01D0FEF7D1
:101A1000BEFD2B68019A1C1213402F4A9B009B5855
:101A20000435FEF796FDA4003F1B380000F01CFBB8
:101A3000284B1B78002B01D0FEF7A9FD2B68019ADB
:101A40001C121340244A9B009B580435FEF781FD6D
:101A5000A4003F1B380002F0F5FE1E4B1B78002B44
:101A600001D0FEF794FD2B68019A1C1213401A4A0C
:101A70009B009B580435FEF76CFDA4003E1B300014
:101A800002F088FF3700134B30601B780437002BBF
:101A900001D0FEF77CFD2B68019A1C1213400E4A00
:101AA0009B009B580435FEF754FDA4003F1B3800F3
:101AB00002F098FE074B1B78002B01D0FEF767FD64
:101AC0002B68019A1C121340034A9B009B58043553
:101AD000FEF73FFD84020020D0A10000FEFFFF7F43
:101AE000A80500208502002004000020A4003E1B61
:101AF000300002F08DFE3700B14B30601B780437A8
:101B0000002B01D0FEF743FD2B68019A1C121340F5
:101B1000AC4A9B009B580435FEF71BFDA300FF1A3F
:101B20003900200000F0FCFEA54B1B78002B01D0F3
:101B3000FEF72DFD2B68019A1C121340A14A9B0051
:101B40009B580435FEF705FDA300FF1A390020005D
:101B500000F06EFD9A4B1B78002B01D0FEF717FDAD
:101B60002B68019A1C121340964A9B009B5804351F
:101B7000FEF7EFFCA300FF1A3900200000F068FD1B
:101B80008F4B1B78002B01D0FEF701FD2B68019ACB
:101B90001C1213408B4A9B009B580435FEF7D9FC5E
:101BA000A300FF1A3900200000F07AFD844B1B7857
:101BB000002B01D0FEF7EBFC2B68019A1C1213409E
:101BC000804A9B009B580435FEF7C3FCA300FE1A15
:101BD00031002000049302F01FFF049B3060FF1AC5
:101BE000774B04371B78002B01D0FEF7D0FC2B6815
:101BF000019A1C121340734A9B009B580435FEF750
:101C0000A8FCA300FE1A31002000049302F01CFF80
:101C1000049B3060FF1A6A4B04371B78002B01D0FD
:101C2000FEF7B5FC2B68019A1C121340654A9B0015
:101C30009B580435FEF78DFCA300FE1A31002000EE
:101C4000049302F0C2FE049B3060FF1A5C4B043721
:101C50001B78002B01D0FEF79AFC2B68019A1C120E
:101C60001340584A9B009B580435FEF772FCA300B2
:101C7000FE1A31002000049302F0C0FE049B306085
:101C8000FF1A4F4B04371B78002B01D0FEF77FFC67
:101C90002B68019A1C1213404A4A9B009B5804353A
:101CA000FEF757FCA300FF1A3900200000F0DAFD10
:101CB000434B1B78002B01D0FEF769FC2B68019A7F
:101CC0001C1213403F4A9B009B580435FEF741FC11
:101CD000A300FF1A3900200000F00AFD384B1B78E2
:101CE000002B01D0FEF753FC2B68019A1C12134005
:101CF000344A9B009B580435FEF72BFCA300FE1AC8
:101D000031002000049300F021FE049B3060FF1A94
:101D10002B4B04371B78002B01D0FEF738FC2B68C7
:101D2000019A1C121340274A9B009B580435FEF76A
:101D300010FCA300FF1A3900200000F079FD204BB1
:101D40001B78002B01D0FEF722FC2B68019A1C1295
:101D500013401C4A9B009B580435FEF7FAFBA30076
:101D6000FF1A3900200001F005FF154B1B78002BEE
:101D700001D0FEF70CFC2B68019A1C121340114A8B
:101D80009B009B580435FEF7E4FBA300FE1A3100CC
:101D90002000049301F0EEFE049B3060FF1A084B14
:101DA00004371B78002B01D0FEF7F1FB2B68019A5A
:101DB0001C121340034A9B009B580435FEF7C9FBD5
:101DC00084020020D0A100000023F7B55A1E019222
:101DD000002B07DA00F0EEFD02F084F902F0DCFAE5
:101DE0006423019300263000194B1968B14212DDBB
:101DF000184B1A6801328A420FDAF0241A601D6803
:101E0000154F6C43E35D002B1FD0E419022B06D164
:101E10002000FEF77DFB019BD8E70022EDE7012BB8
:101E20000DD1002801D100F035F8F0226A43BB182B
:101E30005B680A49C31A8B4201D80223BB54F023C2
:101E40005D43054BEB5C022BE2D00136CCE7C0468C
:101E5000AC05002000000020101200209F86010029
:101E60000020704700207047002070470020704716
:101E700001220020054B06491A61585004310330F5
:101E800058500831801858501A6070470080004040
:101E9000040500000122034B1A64A822D2009858BE
:101EA0007047C0460080004010B5FFF7F3FFFA21ED
:101EB000890005F001F810BD0048704750A40000EB
:101EC0001A20704770B5054E0400335C0D008B423C
:101ED00002D003F0DBFC355570BDC046B0050020D4
:101EE00070B50024064D635D012B05D10021200053
:101EF00003F0CCFC0023635501341A2CF2D170BDE1
:101F0000B005002070470D20704735207047000055
:101F1000F8B501240B6806000D00234204D10D2002
:101F2000FEF7D8FA2000F8BD5B102000052BFAD888
:101F30000E4A9B009C580E4F3B5D002B05D00021A4
:101F4000200003F0A3FC00233B55012E06DD6B6847
:101F5000042B03D10221200003F098FC200003F0A1
:101F600043FB012440002043DDE7C04638A40000C5
:101F7000B0050020F8B501260568354202D0446856
:101F8000344203D10D20FEF7A5FAF8BD6D10192DCE
:101F9000FBD80A4F7B5D012B04D03100280003F0F1
:101FA00075FC7E55064964108C4202DCE143C9177A
:101FB0002140280003F09EFBE7E7C046B005002063
:101FC000FF03000070B501240D68254204D10D20E7
:101FD000FEF780FA200070BD6D10192D17D800246F
:101FE000012804DD4C68043C63425C416400094EF6
:101FF000735DA34204D02100280003F047FC745510
:10200000280003F077FC03000420012BE3D000201C
:10201000E1E7C046B005002070B504000D001928A6
:102020000ED8084E335C012B04D0012103F02EFCA6
:1020300001233355290020004D1EA94103F044FC23
:1020400070BDC046B0050020036810B5DA0703D4A0
:102050000D20FEF73FFA10BD4168581004394A427E
:102060005141FFF7D9FFF6E737B569460A00064B3D
:1020700030CB30C203680220042B02D100F0E8FA12
:1020800037BD00F00DFBFBE710A4000010B5084CB5
:10209000237D002B05D00021142003F0F7FB002343
:1020A0002375142003F026FC43425841800010BDE4
:1020B000B005002010B5084CA37D002B05D00021F1
:1020C000162003F0E3FB0023A375162003F012FC97
:1020D00043425841800010BDB00500207047704752
:1020E00010B5034A0421034801F030FD10BDC0467D
:1020F00018A4000014AB0000E12170B54902144897
:1021000003F06AF8FFF7B4FE0A2003F067FA002331
:10211000FF21104A995401331A2BFBD101220020D0
:102120000D4B01001A6004230C4A0D4D1468002C5D
:10213000FCD02C680002013B20431160002BF5D13C
:102140000122084B1A6003F003FA00F07FFD70BD16
:1021500098110020B005002000D0004000D10040C0
:1021600008D5004004D00040F8B50B4E0700300001
:102170000D0003F079F80400A84200DD2C003D00BA
:10218000EB1B9C4205DD300003F078F82870013528
:10219000F6E72000F8BDC0469811002010B50100F8
:1021A000014803F021F810BD9811002010B5054C2E
:1021B000200003F027F8E1212000490203F00CF889
:1021C00010BDC04698110020064B01201A68064B2E
:1021D00006491A6000239A0001338850642BFAD113
:1021E0007047C046D4050020CC050020682300209D
:1021F00000B59BB00200054901A807F007F901A846
:1022000001F08AFE02F0C8F8FCE7C046D6A4000040
:1022100037B5184D04002868002801D006F0E4FC0A
:10222000A400200006F0D6FC2860002802D1124845
:10223000FFF7DEFF01AB984207D2104B02196B4447
:102240000193934201D20E48F2E7042802D80830E5
:102250002860083C2B680B4A1C1913600A4B0120AC
:102260001C60002309499A0001338850642BFAD17D
:1022700037BDC046D40500207CA400001CFCFFFF35
:10228000ACA40000CC050020D0050020682300206D
:1022900070B50D4D0D4E04004B1C28689B00366830
:1022A000C318B34203D90A20FEF714F970BD2B609E
:1022B0000500AB4205D80F2309011C4021430160F2
:1022C000F4E704C5F5E7C046CC050020D0050020A2
:1022D0000322CB1C70B50C00D9171140C91805009A
:1022E000891000220420FFF7D3FF0023A34206DB5E
:1022F000E343DB171C4000230419237170BDE95C24
:10230000C21811710133F1E710B5830706D1042813
:1023100004D90F2208C81340042B03D00E20FEF767
:10232000D9F8014810BDC046E6A4000010B501244C
:102330000B681C4016D05C10200005F0DBF80B4940
:1023400004F0A6FF06F06EFB03F018FC0022084B19
:1023500005F03EFD03F0BAFB06F0F4FA430001205D
:10236000184310BD0D20FEF7B5F8E5E7D302373965
:102370000000D04010B503240868044006D10428AA
:1023800004D90F2302681340042B03D00E20FEF75C
:10239000A1F810BDFFF7B8FF03782100233B5A4294
:1023A00053411022C01807F001F980239B05C21881
:1023B000044B9A4201D91420E9E743000120184355
:1023C000E7E7C046FFFFFF3F10B5034A022103487D
:1023D00001F0BCFB10BDC046ECA40000E7A4000067
:1023E0000020704710B51E20FEF774F810BD10B520
:1023F0001E20FEF76FF810BD10B51E20FEF76AF81C
:1024000010BD10B51E20FEF765F810BD10B51E20DA
:10241000FEF760F810BD10B51E20FEF75BF810BD8A
:1024200010B51E20FEF756F810BD10B51E20FEF7A1
:1024300051F810BD7047000010B5034A0921034848
:1024400001F084FB10BDC0460CA5000054A500009F
:102450000120034B1860034B1B68834018437047EF
:10246000F8050020D8050020F0B5EFF31081012316
:10247000194083F31088134C134AA4461268134E74
:10248000013A9340124F134A002B17D014680342AD
:102490000FD03D682C60C046C046C046C046C0460E
:1024A000C046C046C0460C4C1568246825605B08D1
:1024B000EAE765462C6014683460F8E781F3108819
:1024C000F0BDC04608050050080000200C05005073
:1024D000E4050020EC050020E005002030B585B0C3
:1024E00001AD0C220649280006F088FB0024285D77
:1024F00001210134FFF7E6FC0C2CF8D105B030BD0A
:10250000E0A50000F0B585B06A463C4B3C4913801D
:102510000F2301AF93700C310922380006F06EFBD7
:10252000FFF7C2FC374B384DC0182B68984201D2D8
:1025300000232B602C68002C44D13E5D012130002B
:10254000FFF7C0FC01340121300003F0BDF9092C74
:10255000F3D100246B461E5D01213000FFF7B2FC71
:1025600001340021300003F0AFF9032CF2D1C82070
:1025700080000138C046C046C046C046C046C0467E
:10258000C046C046C046C046C046C046F1D1002144
:102590000520FFF797FC6B4600211878FFF792FCA7
:1025A0006B4600215878FFF78DFC6B460021987828
:1025B000FFF788FCFFF778FC002413302860200028
:1025C00005B0F0BDFFF770FC2B6800249842F6D3ED
:1025D000052003F009F80D4B0D4EC0180BD43060E8
:1025E0003068032104F0F2FC00230A4A30602B60BB
:1025F00013600124E3E73460F2E7C0460D0E0000EB
:10260000E0A5000010270000F0050020C8FEFFFF35
:10261000D8050020F805002010B50124044002D0A0
:102620004410200010BD0D20FDF754FFF9E7000015
:102630000022054B10B51A60044B1B68934201D071
:1026400002F078FA002010BDF4050020BC10002034
:1026500070B508680D00FFF7DFFF04006868FFF73A
:10266000DBFF621E0100042A14D8451E042D11D878
:1026700005236B439B18012215009D402B00064843
:1026800005682B430360054B1B68002B02D020001C
:1026900002F051FA002070BDF4050020BC100020AB
:1026A00070B508680D00FFF7B7FF04006868FFF712
:1026B000B3FF621E0100042A13D8451E042D10D852
:1026C00005236B439B1801229A40074803689343F4
:1026D0000360064B1B68002B03D00022200002F091
:1026E0002AFA002070BDC046F4050020BC1000206E
:1026F000F0B5050089B008680C00FFF78DFF069063
:10270000022D36DD6068FFF787FF0190A068FFF7B4
:1027100083FF04000127231D661E0793731C029389
:10272000079B9E4235D0052373430593019B019D72
:1027300005330493049BAB421ED0042E16D86B1EA7
:10274000042B13D80122059B2349013B5B199A40B6
:102750009446224A0B681068069A3A4003920DD0BC
:1027600062461A430A60012200280DD17F0001351C
:10277000E0E701240194CDE7029ECFE76246934350
:102780000B600028F2D0039A0299280002F0D3F9D6
:10279000ECE7019B1E1D042E1AD8012C18D1002530
:1027A00005273B0021006B439B1999400B000A4A07
:1027B000013511689943094B11601B68002B05D046
:1027C000019B0022581D290002F0B5F9052DE8D122
:1027D000002009B0F0BDC046F4050020BC10002068
:1027E00010B5041E10DA1A240A4BA400E258012383
:1027F0009340094A09491360094A1160094A0A4984
:1028000011600A4A136010BDFFF75AFBA042EADDCF
:10281000EAE7C04654B20000EC050020080500506D
:10282000E4050020E00500200C05005018050050CC
:102830000200086810B5C3070FD540101823012AFD
:1028400003DD4A68042A00D10833054A1360FFF704
:1028500059FBFFF7C5FF002010BD01204042EDE706
:10286000080000202B4BF7B51B680C00002B03D190
:1028700001204042FFF7B4FF0126246834421AD0F9
:10288000FF226310120260121040DAB21043FF22DE
:102890001B021204134018431F4B1B68202B06D148
:1028A000B4401E4BA40EA400E35800021843FFF7E7
:1028B000DBFD0020FEBD03252540FAD1042CF8D90C
:1028C0000F2322681340062BF3D1FF27130901932E
:1028D0003F02019B9D42ECDA0135AB00E3583342E5
:1028E000F7D05A105812D1B238400843FF211202D3
:1028F00009040A401043084A1268202A06D15B00E6
:102900009B0E06499B00020258581043FFF7ACFD8E
:10291000DFE7C046EC05002008000020D0A700003B
:10292000086810B5C30703D5FFF776FE054B18609E
:10293000054B1B68002B03D0024B186802F0FCF813
:10294000002010BDF4050020BC1000200868F8B578
:10295000C3071AD5FFF760FE0300203B5E2B25D886
:102960000520012258430023114E451DA84219D0CD
:1029700005211024375C3C4200D09B1801395200DD
:1029800064100029F7D10130F0E783070ED1042845
:102990000CD90F2203681A40042A07D11B0905D05D
:1029A0000079D9E701205B001843F8BD0120FCE75E
:1029B000F5A500007FB5A04C2368002B0AD19F4AE3
:1029C0001268002A06D19E4B1B68002B01D0FFF72E
:1029D00099FD7FBD9B4D2A68002A26D1984A12682E
:1029E000002A1BD0FFF78EFD0028F2D0FFF776FDFE
:1029F000924B24681A681C60002A16D0002C14D14F
:102A000001AD0C229049280006F0F8F8285D00215D
:102A10000134FFF757FA0C2CF8D1DAE7874A12682D
:102A2000002AE5D1002BE3D0E0E700210D2002F0E1
:102A30004BFF00210E2002F047FF00210F2002F083
:102A400043FF2E68012E5DD0022E00D1A2E0002EA1
:102A500051D101363100794C04202368994302F0AA
:102A600033FF04212368052019404B42594102F0ED
:102A70002BFF10212368062019404B42594102F0D8
:102A800023FF80212368090119404B4259410C2042
:102A900002F01AFF80212368090219404B42594174
:102AA0000B2002F011FF80212368490219404B429C
:102AB00059410A2002F008FF802123688902194049
:102AC0004B425941092002F0FFFE80212368C902D0
:102AD00019404B425941082002F0F6FE802321683C
:102AE0001B0319404B425941072002F0EDFE310013
:102AF0000D2002F0E9FE2B680321581C04F04CFB6A
:102B0000296066E702214D4C0720236819404B429B
:102B1000594102F0D9FE0820216801404B42594139
:102B200002F0D2FE80212368C90019404B4259416E
:102B3000052002F0C9FE80212368490119404B425B
:102B40005941062002F0C0FE80212368C9011940C6
:102B50004B425941042002F0B7FE802123688903CB
:102B600019404B4259410A2002F0AEFE80232168F1
:102B70001B0419404B425941092002F0A5FE3100C7
:102B80000C2002F0A1FE31000B2002F09DFE31006E
:102B90000E20AEE72021294C0720236819404B4224
:102BA000594102F091FE40212368082019404B4210
:102BB000594102F089FE80212368092019404B42C7
:102BC000594102F081FE80212368490019404B429F
:102BD00059410A2002F078FE8021236889001940BB
:102BE0004B4259410B2002F06FFE8021236889017E
:102BF00019404B4259410C2002F066FE80212368A7
:102C0000490319404B425941062002F05DFE8021E4
:102C10002368C90319404B425941042002F054FE75
:102C2000802321685B0419404B425941052002F082
:102C30004BFE01210F205CE7F4050020E805002091
:102C4000F8050020DC050020E0A50000012010B5FB
:102C50004042FFF7C5FD0020FFF706FC10BD000055
:102C600010B5034A0921034800F070FF10BDC046AB
:102C7000D0A8000018A9000030B502248025094B17
:102C8000094AED009C505C59002CFCD0A124E400C2
:102C9000884202D30021995030BD8025ED001851A3
:102CA0004019F5E700E001400405000010B50028D8
:102CB00006D1C020B02140028902FFF7DDFF10BD20
:102CC000B02080218002C902F7E70000434258414A
:102CD000064B40421840B0239B02C01803680020F6
:102CE0001A0E532A01D11B02180A704700C0FEFFBA
:102CF00030B501248025054B054AED009C505C59F8
:102D0000002CFCD001600021995030BD00E0014052
:102D10000405000043425841074B40421840B0238D
:102D20009B02C018A62310B50902DB05090A194346
:102D3000FFF7DEFF10BDC04600C0FEFF70B50124E6
:102D400080250D4B0D4EED009C515C59002CFCD0A4
:102D5000002902DC00229A5170BD557814782D02AA
:102D600025439478013924042543D4780432240679
:102D70002C4310C0ECE7C04600E001400405000011
:102D800070B505004B680A009C1C2100A400FFF7E9
:102D9000D5FF281970BD0000134B1B68002B0CD009
:102DA0008022B023D2029B0200280BD11A1D5B683F
:102DB0001B0E522B00D110007047B022C02392028C
:102DC0005B02F1E782420DD903681B0E522B09D139
:102DD000436802339B00C018824203D903681B0E6C
:102DE000522BE9D00020E7E7FC06002070B5002058
:102DF000FFF7D2FFFF260500002801D1280070BD93
:102E000003681C143440FFF7C7FFDA2CF4D1050027
:102E1000F2E700008022F0B55200A1B0002167481F
:102E200005F0F5FE802200215200654805F0EFFE16
:102E3000644BFF271B681A00049353425A41100049
:102E40000592FFF733FF049C0020631E9C415E4BFC
:102E500064421C405D4BE418FFF7C8FF0600002EDB
:102E60002DD10498FFF732FF411C0598FFF752FF60
:102E7000059A574D534B2C601A60FFF797F9514B49
:102E800064201B68A0215A4253414F4A5B421340C1
:102E9000B0222C6892029B18E41A6043490204F0A5
:102EA00095F8A0225202030000924A49220007A886
:102EB00006F0ACFA07A801F02FF821B0F0BD326897
:102EC000131412123A403B4003921A000A3A092A9C
:102ED00049D83A4B039A995C002931D110223E48D7
:102EE00005F095FE35002B6803991A123A4091427D
:102EF00009D11A143A400B2A27D0132A2DD00A2AB6
:102F000001D1354B1D602800FFF746FF051EEAD1B1
:102F1000314B196800290FD02000FFF731FF040062
:102F20002D4B5B195968002903D02000FFF728FFBB
:102F3000040004350C2DF3D1204B0121039A995440
:102F40003000FFF729FF060089E73B40022BDADC5F
:102F5000214A9B00D3185D60D5E7102200211E484E
:102F600005F055FECFE71A00153A082AE8D8144AAA
:102F70000399525C002AE3D13500152B00D01500CF
:102F8000300003681A143A40152A0FD01D2A00D1C8
:102F90000025FFF701FF0028F3D1002D04D0200009
:102FA0002900FFF7EDFE0400054BC6E7039A1B124C
:102FB0003B409A42EDD10500EBE7C046FC050020FE
:102FC00004070020FC06002000C0FEFF04C0020031
:102FD00000070020B1A90000F8240020F0B500206F
:102FE000B7B00024FFF7D8FE270005002600002D0B
:102FF0002ED1284D2868FFF769FE32003B00019072
:103000000094254904A806F001FA04A800F084FF02
:10301000224B64201C682B68A0215A425341204A4D
:103020005B421340B02292029B18E41A60434902AB
:1030300003F0CCFFA02252020300009219492200A3
:1030400004A806F0E3F904A800F066FF37B0F0BD6D
:10305000FF226B6829689C460233FF180B12013669
:1030600013409C4200DA1C00FF200A140240039225
:103070006246014001920091039A0B4904A806F0B0
:10308000C5F904A800F048FF2800FFF785FE0500F9
:10309000ADE7C046FC06002022AA00000007002081
:1030A00000C0FEFFCCA900000EAA000070B50020F1
:1030B000FFF70CFE04000120FFF708FE844200DA4F
:1030C00004000A4B1D686A42554128001D60FFF745
:1030D000EDFDA0226B4252021340054A28009B18C6
:1030E000044A611C1360FFF715FE70BDFC0600204A
:1030F0000480010000070020F8B50020FFF7E6FD7E
:1031000007000120FFF7E2FD3E00204D0643204C62
:103110000DD18021C020C9024002FFF7ADFD012181
:103120003000FFF7F7FD1B4B2E6023601DE0874248
:1031300009DD0023B0212B60164B89022360236830
:103140000020012517E0012380212B60124BC902CA
:103150002360F4E7120E522A08D0002800D0236022
:103160000E4800F0D9FEFFF7A1FFF8BD28005A680D
:10317000023292009B188B4205D21A68561CE9D184
:103180000028F2D0D1E72160EFE7C046FC0600201E
:10319000000700200480010004C00200E7A900002D
:1031A000F0B585B0039203220333DC17294D144098
:1031B000E4182B68284F5A42534180225B42D202C6
:1031C000A4103B409B18A21C0291244E9100009138
:1031D0000190316800980A18934215D2FFF71AFE41
:1031E0002B685A42534180225B421F40D202BF18D3
:1031F0003368009A9B189F4206D2194800F08CFE53
:103200000025280005B0F0BD029B356819066B4605
:103210001A7BA423DB051343FF222F00090C19435B
:10322000019B12041B04134019432800FFF760FDA3
:103230000837281D21003760FFF75AFD002C04D005
:103240000A9A21003800FFF779FD009B083BFF1820
:103250003760D6E7FC06002000C0FEFF0007002014
:103260008BA9000010B5FFF7D5FD10BD70B59AB061
:10327000FFF742FFFF221E4CD2000021200005F084
:10328000C6FCFF25FFF7B2FD0026002814D102007E
:10329000C300E3580130591E8B41D218FF28F7D1E3
:1032A000144901A806F0B2F801A800F035FE124852
:1032B00000F032FE1AB070BD03681A142A400A2AC0
:1032C0000AD11A122A40FF2A03D0D200A1180B718A
:1032D000A050FFF761FDD8E7132AFAD11B122B404B
:1032E000FF2BF6D0DB00E2181671E650F1E7C0467E
:1032F000701B002057AA00006BAA00000021094B98
:10330000094A59600131516059680029FCD00021F7
:103310001961012393600222044B8131FF315A501D
:103320001A607047FC1000400010004000E100E00F
:103330000222064B0121DA670022054B5A61054A39
:1033400011615A69002AFCD07047C04604E100E0D0
:10335000FC1000400010004010B5044C2378002BF6
:1033600001D0FFF7E5FF0020207010BD0508002008
:103370000120024B1B685B0018437047880800203F
:1033800003480368002B02D11422037102607047C6
:10339000202500200120024B1B685B00184370476A
:1033A0000C00002070B504000D001600FEF77CFD37
:1033B0008023012200215B055B6E6270E270020ACD
:1033C000A271020CE2711A0A60716372000EA2729D
:1033D0001A0C1B0E26702571A1702072E2722373E5
:1033E00070BD0000124B10B51B68124C5A1C0FD058
:1033F000114C002B0CD0114C012B09D0104C022B7E
:1034000006D00D4C042B03D00E4C052B00D10B4CD9
:1034100021000D4806F024F8200006F029F80300EA
:10342000042204339B0809481B011343036010BDA9
:1034300010000020F3AA0000ECAA0000FEAA000081
:1034400003AB0000F8AA00000C250020082500208E
:1034500070B5214C2278002A3DD1204B01215A60C1
:103460008022D20511605A68002AFCD00022072071
:103470001B4B1C4901255A500439585008315A50E9
:1034800019481A4958501A491A485A501A495A5054
:10349000A622D2009D50082218495A500431585093
:1034A00002201749585017491748585017480439EF
:1034B0005850182016495850C12189005A500539D2
:1034C000FF395858921802435A501249124A9950DB
:1034D000FFF714FF257070BD05080020FC000040B8
:1034E000001000400C050000746962751C050000A6
:1034F00024050000200004022C0500001405000033
:10350000340500003C050000FFFF00002110010011
:1035100054050000060800200405000070B50E4B9D
:1035200006001B78002B01D1FFF792FF00200B4D06
:103530002C7884420ED00A4B202219780323091BD1
:103540001940084B4901C918300005F057FB01200C
:10355000013C2C7070BDC046050800208C0800207E
:103560000408002006080020002330B589B09842E6
:1035700025DD03240D682C409C4220D12300042D1E
:103580001DD90F212A681140062918D112091F2AB6
:1035900015D96846FFF7C2FF230000280FD06B46FD
:1035A000012218781300A04203DB6B461B5D5B0011
:1035B00013430134A1006B50202CF3D104231800D5
:1035C00009B030BD70B5414B8AB01B78002B01D1DA
:1035D000FFF73EFF02AD2800FFF7A0FF002802D151
:1035E00000200AB070BD2B780B2BF9D96B78012B1A
:1035F000F6D1EB78012BF3D10023354E354C3360F7
:1036000023712B79344A1360002B0ED115216944A4
:103610004A780B7812021A438B781B041A43CB7832
:103620001B0613433360002318E0012B20D1152122
:1036300069444A780B7812021A438B781B041A43A8
:10364000CB781A211B06134333600E236A7C69442E
:10365000934200DD130000229A4232D1042000215F
:10366000E21804339B101B01034311712360B8E778
:10367000022B03D16A7B10331621E8E7042B0DD10E
:10368000152108226944684605F0B8FA00980199A6
:1036900002F08CF905F056F93060C4E7052BC2D171
:1036A000152108226944684605F0A8FA0098019996
:1036B00002F07CF905F046F930606A7D0A231E218C
:1036C000C5E78D5CA01805710132C5E7050800202B
:1036D00088080020202500201000002010B5134B82
:1036E00004001B78002B01D1FFF7B2FEFFF720FE8C
:1036F00000200F4A0F49104B5450586001301060A1
:1037000058680028FCD000201861013090601869CA
:103710000028FCD0094B0A481B785B011B1853504A
:10372000FFF706FEFFF7EAFD10BDC04605080020C2
:103730000010004004050000FC10004004080020B8
:103740000608002030B589B000281EDD03230A6872
:1037500013401AD1042A18D90F20116808400628EE
:1037600013D109091F2910D9012401339900515897
:103770000020214201D04910C8B26D46591E68543C
:10378000202BF2D16846FFF7A9FF002009B030BD19
:1037900010B5002813DD0C68E30710D56410532C16
:1037A0000DD8084B1B78002B01D1FFF751FEFFF716
:1037B000BFFDA123044ADB00D450FFF79FFD00208A
:1037C00010BDC046050800200010004010B50028BC
:1037D0000EDD0C68E3070BD56410FF2C08D8054BF1
:1037E0001B78002B01D1FFF733FE034A034BD45063
:1037F000002010BD05080020001000402405000036
:1038000013B5002814DD0C68E30711D5094B6410CB
:103810000093094B0193072C0AD8084B1B78002B07
:1038200001D1FFF715FE6B46054A1957054BD150DC
:10383000002016BDE2ECF0F4F8FC000405080020BE
:10384000001000400C05000070B588B0002820DD95
:103850000324086804401CD104281AD90F230268E5
:103860001340042B15D1FEF74FFD060005F000FEB6
:103870000500122800D912252A0002210D326846BF
:10388000FFF790FD6B465D73A54205DC6846FFF7C8
:1038900025FF002008B070BD2300325D6B449A7391
:1038A0000134F1E7F0B50D008BB0012831DD0324C0
:1038B000086804402DD104282BD90F230268134037
:1038C000042B26D14B68DB0723D5FEF71DFD6E6860
:1038D00007007310019305F0CBFD05000E2800D9F9
:1038E0000E252A000121113202A8FFF75BFD6A466E
:1038F000127902AB5A7302AA73129373019B761466
:103900001B0ED67313745574A54205DC02A8FFF78D
:10391000E5FE00200BB0F0BD3A5D02A963189A7471
:103920000134F1E730B589B0002814DD0C68E307F5
:1039300011D5102268460021FFF734FD6B466A4618
:1039400065105D73684663122D0E64149373D4730F
:103950001574FFF7C3FE002009B030BD174B184A9D
:103960005968002903D0002159600131916019691B
:1039700000291FD0002018618023DB00D358114993
:10398000012B18D1A923DB00D3585B420B600E49F1
:103990000B78032B01D801330B7003200B490B78F4
:1039A000013303400B700A495B015B18094953500E
:1039B0000123936070470860FAE7C046FC1000409E
:1039C000001000400C0000208C080020040800209B
:1039D000060800200405000010B5034A0E21034824
:1039E00000F0B4F810BDC0467CAA000073AA000025
:1039F000044A05491368C85401339B059B0D1360A5
:103A00007047C046A80C0020A808002070B5114CD3
:103A1000114A2368834202DC0023236016E0155C10
:103A2000411C2E00FA3E012E05D899420FDA555C52
:103A3000013D1F2D01D90800ECE70100151A565C65
:103A40006E5401318B42FADC181A206070BD15707B
:103A5000FAE7C046B4100020B40C002010B5FEF701
:103A600019FA064B1A68824201D900221A601B68B3
:103A7000C31A034898428041404210BDA408002068
:103A8000204E000010B5094C094A23681268934281
:103A900000D110BD074AD05CFEF780FB0028F8D0AB
:103AA000236801339B059B0D2360ECE7AC0C0020E1
:103AB000A80C0020A808002010B50400064B074AF7
:103AC0001B6812689B1ADB439B059B0DA34200DB1E
:103AD00010BDFFF7D7FFF1E7A80C0020AC0C0020C9
:103AE000F7B5050056680191B000441C0630170078
:103AF000FFF7E2FFFB20FFF77BFF1C20FFF778FFBB
:103B0000E8B2FFF775FFE0B22412FFF771FFE0B2F1
:103B1000FFF76EFF6B461879FFF76AFF0025AE428C
:103B200000DCF7BDAB00FB189C680135E0B2FFF785
:103B30005FFF2012C0B2FFF75BFF2014C0B2FFF797
:103B400057FF200EFFF754FFE9E7000070B5074E5E
:103B50003368092B08DC0C255D43054C01332851E3
:103B600064196160A260336070BDC046B00C002073
:103B700044250020F0B587B002900C00012803DC3A
:103B80001B20FCF7A7FC45E0244B08680093830743
:103B900009D1042807D90F2302681340042B02D14E
:103BA000FEF7B2FB00901D4B60680193830709D1BB
:103BB000042807D90F2302681340042B02D1FEF713
:103BC000A3FB01900027164B1B680493049BBB4288
:103BD000D6DD0C267E43134B0099F618306805F0AD
:103BE00035FC051E05D17368B6680593059B9D429B
:103BF00001DB0137EAE730680199039605F026FCFE
:103C00000836002808D121000298039B08310238A9
:103C10005B68984707B0F0BD0135E7E7E6A4000010
:103C2000B00C00204425002010B5FFF719F8FEF76E
:103C300057FAFEF7C9FBFEF7FFFBFFF7CDFE00F0DA
:103C4000F5FD00F07BFF10BD962210B5120100219A
:103C5000034804F0DCFF0022024B1A6010BDC0468E
:103C600010120020AC050020064B074A1B681268A2
:103C70009B1ADB439B059B0D0122834200DC002243
:103C800010007047A80C0020AC0C0020F8B505000F
:103C90000C0016001F1E0ED10320FFF7E5FF0028C1
:103CA00008D0FA20FFF7A4FEE8B2FFF7A1FEE0B2C9
:103CB000FFF79EFEF8BD501DFFF7D6FF0028F9D094
:103CC000FB20FFF795FEE8B2FFF792FEE0B2FFF7A8
:103CD0008FFEF0B2FFF78CFE3012C0B2FFF788FE05
:103CE0003C00E31B9E42E5DD2078FFF781FE0134B6
:103CF000F7E7000070B50024F0250B4B1B68A342CA
:103D000002DCFFF7A1FF70BD2B006343074A9B183D
:103D10001A78002A05D05978002311201A00FFF7DD
:103D2000B5FF0134E9E7C046AC05002010120020C1
:103D3000F8B507000024F0252B0063430C4A01343A
:103D40009E18B74211D0317800290BD00133D15CD5
:103D5000002311201A00FFF799FF2A0000213000EC
:103D600004F055FF0A2CE7D1F8BD024B1C60F9E7BF
:103D700010120020AC050020F0B504001000012254
:103D80000300FFB00D00134013D06B461A706A4653
:103D900069464310537042121B0E8A700B71052244
:103DA0006B464014C87029002000FFF76FFF7FB0FA
:103DB000F0BD032606401ED104281CD90F2201683D
:103DC0000A40042A29D102236A461370FEF79CFA9E
:103DD000070005F04DFBF823FF33984200D9180087
:103DE000B04202DC421C6B46DDE76A460136731EB8
:103DF000FB5C9355F4E7042801D0002809D16A46FA
:103E0000032304381370424250416B46022258701B
:103E1000C9E7002ECBD10428C9D90F21026811406F
:103E2000052913D16E4601393170F8211209FF318D
:103E300092008A4200DD0A00934201DB0132D2E7A0
:103E40006E460133C118C978F154F5E70629AED1A1
:103E50001209642A00D964226E46052131700136A8
:103E60009A4202DC05235A43E8E70127013399000F
:103E7000415839420BD03941012737700F12717008
:103E8000B7700F14090EF77031710536E8E7014974
:103E9000F2E7C04619FCFFFF70B502000024F021D4
:103EA0000D4E0800604380194578954203D00134D7
:103EB0000A2CF6D170BDF022002104F0A8FE074ABA
:103EC0001368013BA34200D11460002329001A00AB
:103ED0001120FFF7DBFEEDE710120020AC050020FB
:103EE00010B5B2B002236A460400137005F0C0FAA0
:103EF000C72800D9C7200023984207DC421C6B4624
:103F0000FE211420FFF7C2FE32B010BD6946013316
:103F10005A1EA25CCA54EFE730B5B3B002236A461A
:103F20000500137005F0A4FA0400C72800D9C724BF
:103F300000239C420BDC20003230FFF7BDFD621CE9
:103F40006B46FF211420FFF7A1FE33B030BD694658
:103F500001335A1EAA5CCA54EBE70000F7B5234BA5
:103F600006001B68F02100930023009A9A4211DC9E
:103F70000024F0231A006243019201991C4A55184B
:103F80002F78002F12D001340A2CF3D11948FFF7F3
:103F9000C3FF29E00A005A43154882185078B042FE
:103FA00002D11278002A1FD10133DEE7F022390056
:103FB000280004F02CFE02230D4A0199EB605354B3
:103FC0000D4AF1008A58009B6E70AE70AA602F6196
:103FD0006F61A34202DC054B01341C6000233100F9
:103FE0001A001020FFF752FEF7BDC046AC050020B6
:103FF00010120020EDAF0000701B002010B5FFF77D
:1040000079FEFF24084AE3005B429B18074AD35C11
:10401000043B012B03D8E043C0B2FFF79FFF013CF4
:10402000002CEFD110BDC046FC070000701B002023
:10403000F7B50E00FF247F2501901C4AE300D31A38
:104040001B4A9A181278062A01D0032A1DD1FF2292
:10405000D2009B18186883682B401C2B15D1C368AD
:104060001A002A40042A10D102692A40192A0CD1C8
:104070001B0A01339B000C30C018FEF745F90700FE
:1040800005F0F6F90023B04209D0013C002CD4D150
:10409000F7BD019AF95CD25C9142F6D101339E42A0
:1040A000F7DCE043C0B2FFF759FFEEE7701B0020DA
:1040B000FC07000070B50500FF24084AE3005B42DE
:1040C0009B18074AD35CAB4203D1E043C0B2FFF771
:1040D00045FF013C002CF0D170BDC046FC0700003C
:1040E000701B0020F7B5FDF7D5FE514B1A688242D0
:1040F00001D900221A601A684E49821A8A4200D8F1
:1041000083E01860FDF7D0FE071E00D101370020C4
:10411000FDF7BCFF01900020FDF7CCFF019B009054
:10412000454C464D002B14D02368002B00D07AE07C
:104130002B682760002B00D171E0414B01261B78D2
:10414000002B63D10920FFF7B5FF3E4B1E703C4B9F
:104150001E70009B002B12D02B68002B0FD1236800
:104160002F60002B1ED0374B01261B78002B52D11D
:104170000920FFF79FFF334B1E70314B1E702368E1
:10418000002B0FD02F4E3278002A0BD19F4200D245
:1041900027602368FB1A312B04D90720FFF78AFF19
:1041A000012333702B68002B0FD0254E3278002A64
:1041B0000BD1BB4200D92F602B68FF1A312F04D9D5
:1041C0000820FFF777FF012333702368002B0CD002
:1041D000019B002B09D11B4E3378002B02D1072005
:1041E000FFF768FF0023236033702B68002B0CD08F
:1041F000009B002B09D1124C2378002B02D1082000
:10420000FFF758FF00232B602370F7BD0720FFF74F
:1042100051FF0C4B9CE70820FFF74CFFADE7009BDC
:10422000002B9CD1ABE7009A002A95D1AAE7C046A3
:10423000A00800200F270000900800209808002008
:104240009C0800209408002037B500240500FFF7E3
:1042500051FD01A80194FDF707FF21002000FEF7A2
:10426000E7F9FEF7A7FBFDF739FFFDF738FFFEF78B
:10427000EDFCFDF735FEA54204D0FDF7A5FF024891
:10428000FFF74AFE37BDC046DEAF0000002310B581
:1042900001001A001120FFF7F9FC10BD07B56B46AD
:1042A000197069465A7013128B701314120ECB706A
:1042B0000A716B46010005221320FFF7E7FC07BDDA
:1042C00010B50A0001001220FFF756FD10BD70B5B1
:1042D000050008000C003230FFF7EEFB2B00220037
:1042E00000211B20FFF7D2FC70BD10B50C000300AD
:1042F000110014202200FFF7C9FC10BD012370B586
:10430000FF24084A41185B42884201D3D84370BD5C
:1043100006781D0A234073409B009B5801306B4078
:10432000F2E7C046C0AB0000002313B501930B4B6E
:10433000C2000400D058002805D043680830990016
:10434000FFF7DCFF01900920FFF7B6FB01AB042269
:1043500021001720FFF79AFC13BDC046701B0020F8
:1043600070B506000020FEF717FD0024FF25002889
:1043700001D1200070BD03681A142A40152A07D104
:104380001B122B40B34200D10400FEF705FDEEE7FF
:104390001D2AFAD10024F8E7F0B580279DB0FFF779
:1043A00071FBAD4CAD4D2068FF00391A4019FDF787
:1043B000DBFE23680600C3182360002B0ED11DB05E
:1043C000F0BD2068391A2818FDF7CEFE23680600D4
:1043D0001B182360FDF75EFDA14B1860002EF0DC7A
:1043E0002B78FA2B00D013E12368022B07DCFFF7B0
:1043F00035FB0028E3D00120FFF708FBDFE76878F2
:10440000AC78023818281FD802F04CFD0D20242863
:104410002B341E3E6872768CDEEF1E1E1E1E1E1E84
:104420001E1E1E1EFD00FF2C0ED02000FFF734FDC7
:1044300000228C4BE100CA505B181A7121000092D7
:1044400013001320FEF7ACFE0320D5E72000FFF792
:1044500085FDF9E72000FFF71FFDF5E7FFF7CEFD2B
:10446000F2E7FFF747FC0020FFF7EEFE7E48FFF77C
:1044700053FDE9E7632CE7D87C4BA200D25821001A
:104480001520FFF779FCDFE700242000FFF768FF25
:10449000061E03D10134642CF7D1D5E7083004F0AF
:1044A000E7FF05000530FFF707FBFB20FFF7A0FA49
:1044B0001D20FFF79DFAE0B2FFF79AFAE8B2FFF786
:1044C00097FA2812C0B2FFF793FA3700BB1B9D4240
:1044D000E0DD387AFFF78CFA0137F7E700211D207D
:1044E00000910B000A00FEF75BFEFDF76DFEABE7E7
:1044F0002000FFF719FFA7E7FDF7DEFC03AC5C4ADD
:10450000642100905B4B200004F04EFF022320004A
:10451000237004F0ADFF2300020000211620FFF7F6
:10452000B5FB91E700244F4AE300D558002D28D071
:104530006B689E00701DFFF7BFFA2B00002532004C
:10454000083321000120FFF7A1FB0020FEF724FC27
:104550002F002E00002818D1002F04D03A0001218E
:104560002000FFF7BDFA002D04D02A000221200010
:10457000FFF7B6FA002E04D0320000212000FFF72A
:10458000AFFA0134FF2CCED15EE7FF2103681A1287
:104590000A40A24209D11A140A400B2A08D10B4042
:1045A0000CD0012B0CD0022B0CD0FEF7F5FBD1E781
:1045B000132AFAD100252F002E00F6E70600F4E7B3
:1045C0000700F2E70500F0E70024FFF793FB220065
:1045D000210000942300DA20FEF7E2FDFF222100F3
:1045E000D200204804F013FB7FE7012C02D1FEF734
:1045F000F5FC29E7022C02D1FEF734FE24E7012066
:10460000FFF722FE20E7002321001A001A2086E788
:10461000FB2B00D0EFE62268042A00DCE7E62E79C7
:10462000E878154B360206439E4200DDE3E6331D73
:104630009A4200DCDBE6EB5CFE2B00D0DBE66B781D
:10464000AC78711E1B2B6BD018D8012B2BD0082BEC
:104650003DD0701DD0E6C046B4100020B40C002040
:10466000A4080020701B0020C0AF000068230020B9
:10467000D7AF0000D2AF0000F60300001D2B60D0C2
:1046800052D31E2BE5D1012CE3D10029E1DD6B795A
:10469000002B03D01C00322B00DD322464235C434A
:1046A000344B1C60D5E7FF2CD3D02000FFF7F4FB80
:1046B0006D79314AB31E009221002A000A20FEF7CC
:1046C0006FFD2E4BE400E0501B191D71C1E7632CF8
:1046D000BFD86A79022A13D0032A1BD0012AB8D185
:1046E000E979AB79090219432B7AA4001B04194319
:1046F0006B7A1B060B435B001343214AA350A8E7C8
:104700000029A6DDB11E1C48FDF7E2FD1C4BA400EC
:10471000E0509EE7AB79A4005A1E93419B00ECE762
:104720001848FFF785FC94E7FF2C92D06A79022A9B
:104730008FD811490B2000912100B31EFEF730FDE8
:1047400087E70B00632900DD6323002203A893425F
:104750000ADCD9430022C917194041180A700133F5
:10476000009021001520E9E7A91849798154013208
:10477000EDE7C04604000020BA0C0020701B0020AA
:1047800068230020B90C00200120704710B5064CAA
:10479000200000F00BFB0549200000F02FFB012258
:1047A000034B1A6010BDC046E0100020801A0600BE
:1047B000B810002010B501210D20FDF783FB012169
:1047C0000E20FDF77FFB00210F20FDF77BFB044C43
:1047D000200000F027FA1021200000F03FFA10BD61
:1047E000C010002010B504680D20E30703D5641045
:1047F000FF2C03D91720FBF76DFE10BDFFF7DAFF82
:10480000E1B2024800F04CFA0020F6E7C0100020A8
:1048100010B5FFF7CFFF0021034800F041FA430035
:104820000120184310BDC046C010002010B5034A37
:1048300007210348FFF78AF910BDC04604B0000005
:104840003CB00000F8B5012306681E4205D045685B
:104850001D4202D084681C4203D10D20FBF73AFEB2
:10486000F8BD76101520802EF8D86D101620FF2D7B
:10487000F4D86410FF2C01D91720EFE70B4B1B680D
:10488000002B01D1FFF782FF094FF1B2380000F091
:104890004CFBE9B2380000F04FFAE1B2380000F00A
:1048A0004BFA380000F0ACFB0020D9E7B81000202C
:1048B000E0100020F7B501242300A0421BDD0D68A5
:1048C0002C4218D01A4B25411B684C68002B01D193
:1048D000FFF75CFF0127174EE9B2300000F025FB1F
:1048E0003C420AD03C413000E1B200F025FA3000F1
:1048F00000F086FB00231800FEBD03252540F6D1FD
:10490000042CF4D90F2322681340062BEFD113098E
:104910000193019B9D42EADA0135AB00E15839422F
:10492000F7D04910C9B2300000F006FAF1E7C046EE
:10493000B8100020E0100020144B70B51B68050073
:104940000E00002B01D1FFF721FF114CEDB2290021
:10495000200000F0EAFAF1B2200000F0EDF90021A9
:10496000200000F0EDFA002801D0404270BD012285
:104970002900200000F0D4FA200000F0CEF9002831
:10498000FAD0200000F0CEF9F0E7C046B8100020C1
:10499000E010002010B501240368234202D04168D2
:1049A000214203D10D20FBF795FD10BD5810802842
:1049B00001D91520F7E74910FF2901D91620F2E7A0
:1049C000FFF7BAFF40002043EFE710B5072118209A
:1049D000FFF7B2FF7F2801DD0138FF3803007F3386
:1049E00001DA7F20404264235B4258437F2102F07A
:1049F000EDFA012340424000184310BD10B50821D4
:104A00001820FFF799FF0300C00FC01801234010C2
:104A100015304000184310BD10B505211820FFF7D0
:104A20008BFF7F2801DD0138FF3803007F3301DA77
:104A30007F20404264235B4258437F2102F0C6FA44
:104A400043000120184310BD10B503211820FFF7C3
:104A500073FF7F2801DD0138FF3803007F3301DA5F
:104A60007F20404264235B4258437F2102F0AEFA2C
:104A700043000120184310BDF8B5012302001800BF
:104A80009A4236DD0E68334233D003244D682C4001
:104A90002FD1042D2DD90F2229680A40062A28D1AA
:104AA000144B1B68002B01D1FFF770FEEB0704D4F9
:104AB0002B681C09202C00DD20247610F1B20E4E4C
:104AC0002200300000F02CFA0435A700EF19AF42A5
:104AD0000CD0300000F021F90028FAD0300000F0AE
:104AE00021F901234000184301C5F0E701206400CB
:104AF0002043F8BDB8100020E010002000207047CF
:104B00000120704700207047002070470120704747
:104B10000020704700207047002070470020704739
:104B20000020704700207047002070470020704729
:104B300000207047704770477047000010B5034A67
:104B40000E210348FFF702F810BDC04680B00000F8
:104B5000F0B0000010B5FDF7CFFA0648FDF758FB9E
:104B6000FFF762F80448FFF7D7F9FEF77FFBFFF77E
:104B700045FA10BDE204000079B1000010B5FDF760
:104B800023F910BD70B5002504AC24780573A94243
:104B900005D10A4B0A4A23210A4803F0B3FF0160FA
:104BA0000949920052589B0002715B58A40083711E
:104BB0006358856043710223C37170BD91B10000D9
:104BC000F6B100009FB1000054B20000037B002B3F
:104BD00004D143738373036101330373704700008F
:104BE0001FB50191A02100240068C900D2B2445031
:104BF000012A10D0A24209D0032A0AD0074A8350C2
:104C0000074B019AC250012343501FBD0222134398
:104C1000F4E70422FBE70622F9E7C046540500004A
:104C20002405000010B50400FFF7D0FFA12223687F
:104C3000A179D20099506179064A200099502179D2
:104C400004329950044B19685A689B68FFF7C8FFF3
:104C500010BDC0460C050000D41000204BB2002B44
:104C60000FDB80233F290FD81F290FD80F290FD81A
:104C700007290FD803290FD81B060168074A8B5054
:104C8000704780239B04F8E7DB04F6E71B05F4E795
:104C90005B05F2E79B05F0E7DB05EEE72405000086
:104CA0000368074A99501A00FC32D1680029FCD0E9
:104CB000A321C90058580023C0B2D3607047C04632
:104CC0001C05000007B58022074BD2051A600022A0
:104CD0009A6002321A7111230E3200930349053390
:104CE0000348FFF74FFF07BDD410002000300040FD
:104CF000C0100020F8B505000E0017000024BC42CB
:104D000008D02B68315D1B6828009847002801D027
:104D10000134F4E72000F8BD704710B51C3000F0F6
:104D2000A9F910BD10B51C3000F096F910BD10B5F2
:104D30001C3000F0A5F910BD70B5437E0D00002BAE
:104D400001D1002070BD6430040000F0A2F90028F9
:104D5000F7D12000290000F070F90120F2E70000EF
:104D6000F7B50193FA23002504009B0083600D4BE7
:104D70004560083303601C300F00160000F052F944
:104D80002000643000F04EF9074A2761B600B3589E
:104D900020006375019B9B009B586576A576A375E3
:104DA000FEBDC04634B2000054B200000123A02270
:104DB000C375837D0E49C133FF33D2059B009950E3
:104DC000437DC133FF339B009950CC220169094BCD
:104DD0005204CA5005220169243BCA50827D0169F0
:104DE0000833CA500269417D034BD1507047C04619
:104DF0000C060000240500000C050000A022002382
:104E000010B50469D200A3500A4CA1420FD90A4C34
:104E10008C425B4109495B420B40CD21C9045B18C0
:104E200004690749635005210369995010BDCC23DB
:104E30005B04F5E7A086010090D00300000098FD18
:104E400024050000F7B5040000200D000193824204
:104E500065D01600402A00D9402627001C373800AC
:104E600000F0F6F8B1232269DB00D550802201233F
:104E7000216992008B50A27E002A03D1226913621D
:104E8000226913600025731EAB4207D1019B002BE2
:104E900004D08022022123699200995001222369C3
:104EA0001A622369FC33DA68002A02D19A6A002A5E
:104EB000F9D09A6A002A0BD1DA60A3232269DB00B9
:104EC000D1583800C9B2013500F0B7F8B542DAD38D
:104ED000019B2269002B0FD11300FC339B6A002B2E
:104EE0000AD10133A376D3612369FC33DA6C002A3B
:104EF000FCD00022DA640AE000230121A37651618C
:104F00001A002369FC3399680029FCD09A60236950
:104F1000FC339A6A002A01D000229A62E8B2FEBDF0
:104F200010B50123FFF78EFF10BD0300AC3310B5A1
:104F300004001970643000F08BF80123637610BD13
:104F40000023020070B5AC3243760D001178B12217
:104F500004000069D20081508022216992008B50A8
:104F6000226901331362226993602600643630009F
:104F700000F080F8002812D0300000F06DF81E4BD1
:104F80002269D0502369FC331A6A002A02D19A6A36
:104F9000002AF9D09A6A002A01D11A62E5E723694A
:104FA0000122002D0DD11900FC31896A002908D198
:104FB000DA612369FC33DA6C002AFCD00022DA645F
:104FC00007E05A612369FC339A68002AFCD000226A
:104FD0009A6000202369FC339A6A82420BD098625F
:104FE0002169064A8B588B501800022B03D0181FDA
:104FF000431E9841033070BD1C050000C40400002E
:1050000010B50121FFF79CFF10BD000010B5132360
:10501000122202490248FFF7A3FE10BD00400040E3
:10502000E010002010B540220021040003F0EFFD45
:10503000002320002364636410BD10B53F24026C7C
:10504000531C2340446C9C4201D08154036410BD26
:105050000023036443647047436C026C934206D0A0
:105060003F21C25C01330B404364100070470120B4
:105070004042FBE7036C406C181A00D54030704783
:10508000436C026C934201D0C05C704701204042E7
:10509000FBE73F22036C406C01331340181A434274
:1050A0005841C0B27047000003210A4802680A4311
:1050B0000260094802680A4302600849084A094B2D
:1050C0009B1A03DD043BC858D050FBDC00F012F8FB
:1050D000FBF71AF8240500405405004054B70000BF
:1050E0000000002044020020FEE7FEE7FEE7FEE7A6
:1050F000FEE7FEE72D4B10B51A68D2B2012A0FD198
:105100002B4A126812070BD12A4AE0241168F022B8
:105110000800104021422DD12749096811422CD0A6
:105120001A68D2B2012A12D12149096809070ED1A1
:10513000F020204909680140402908D11E4909682A
:10514000014204D18020C121C005C90042501B6822
:10515000DBB2012B0DD1164B1B681B0709D1154B78
:105160001A68F0231A40A02A0FD1134A12681A4273
:105170000ED010BD3028CFD0D2E7104A10491160B0
:105180008021104A09021160CAE7D02AF1D1ECE768
:105190000D4B1A68012A04D00C4A1A601A68012AB9
:1051A000FCD1C0220A4B1A60E3E7C046E00F00F0D2
:1051B000E40F00F0E80F00F0EC0F00F004050040F1
:1051C000DFFF07C0186C004000EC0640759300003C
:1051D00014EC06400120704710B503681322DB6908
:1051E000984710BD70470000054B0269D150036914
:1051F000FC331A6A002AFCD0002201201A62704790
:105200001C050000030010B55C331A781F231A40F8
:105210001E3B19009140114AD167C2220421046942
:105220009200A150026953600269D360A02300225A
:105230000169DB00CA5001230169094A5B428B50B6
:105240000169084A8B5001690C3A8B500169083298
:105250008B501430FFF7FCFE10BDC04604E100E0A7
:105260000C0500001405000010B51430FFF702FF14
:1052700010BD10B51430FFF703FF10BD10B514308A
:10528000FFF7EAFE10BD0000030070B55E331A7828
:105290000469724BE25003005D331A780469704B65
:1052A000E250030061331C7802696E4B012C00D080
:1052B0009EE005005F352E78A225ED0056510200D4
:1052C00060321578A1220669D200B5500269D45027
:1052D0009623DB00994200D88CE096231B0199426B
:1052E00000D88AE096235B01994200D888E0962393
:1052F0009B01994200D885E0E1239B01994200D8A7
:1053000082E09623DB01994200D880E0E123DB01B3
:10531000994200D87DE096231B02994200D87AE09A
:10532000E1231B02994200D877E096235B02994261
:1053300000D874E0E1235B02994200D871E0E123D8
:105340009B02994200D86EE0474B994200D86CE02E
:10535000E123DB02994200D86AE0E1220023120334
:105360008A425B41414A5B421340802252059B18AE
:1053700001693F4A8B50A02304220169DB00CA5017
:1053800000210369FC33D9600369FC3319620123EE
:1053900001690B6001698B60C12104698900625059
:1053A0001F215C3002780A4093406231314AFF315C
:1053B00053500021415600293CDA0F230B40083B93
:1053C0002D4C9B089B001B1903242140A140FC3459
:1053D0008C40DD69A5432C00C0258D402900214368
:1053E000D9611F23017819401E3B8B40136070BDAB
:1053F00000246CE79E23DB02BAE79D231B03B7E77B
:105400001E4BB5E71E4BB3E7EC239B03B0E71D4BE8
:10541000AEE71D4BACE71D4BAAE71D4BA8E71D4BA4
:10542000A6E71D4BA4E71D4BA2E78023DB049FE703
:105430001B4B9DE78C080F4BA400E41803230B4083
:10544000FF21C025DB009940AD0066598E43310035
:10545000C0269E4033000B436351C2E70C05000099
:10546000140500006C05000090D0030000D0BEFEC3
:105470002405000000E100E000ED00E000B01300B2
:105480000050270000A04E0000F0750000509D0065
:1054900000F0EB0000903A0100E0D70100B0AF034C
:1054A00000705F07F7B5009308AB1B7800250193E8
:1054B000FA2304009B0083600E4B456008330360B1
:1054C00014300F001600FFF7ADFD23005C33276199
:1054D0001E70009B084A9B00995823005D33197089
:1054E000019B20009B009A5823005E33DD701A70E8
:1054F000FEBDC046D0B2000054B20000036910B532
:105500001A00FC32D2680400002A0AD0A322D2007A
:1055100099581430C9B2FFF790FD00222369FC337B
:10552000DA6010BD10B50248FFF7E8FF10BDC046B5
:10553000981100201D2307B5022200930249013370
:105540000248FFF7AFFF07BD002000409811002080
:1055500010B5002801D003F0BFFE10BD7047000059
:1055600010B500F011F8FFF7F9FF012000F000FA84
:10557000FFF7F0FAFFF702FB024B002BFAD000E036
:1055800000BFF7E700000000C420114B80001A584C
:1055900010491140C02212020A431A50C021802231
:1055A000490092025A501A608023A3220021DB0591
:1055B000D20099500122F9309A60074BFF30195000
:1055C000C120023180001950403019501A607047D4
:1055D00000E100E0FF00FFFF00100140014B1860F8
:1055E0007047C0465C000020F7B500231E285AD83B
:1055F000384B8000C258042A5BD007D8022A54D006
:1056000055D80423012A09D000234CE0062A54D09F
:1056100051D31A2A53D002231B2AF5D12E4A1168DE
:1056200008294ED909294FD00A240226A020012595
:105630002A4AC00015502A482A4D07681C20BF007E
:1056400007402948019700685759009027481B02D6
:1056500007401F43C02300989B020340FF2057517F
:105660005759000207401F43019B1F43009B5801ED
:105670006023184007433E43565101251C4B1560DB
:1056800058680028FCD000205860A1230125DB00C9
:10569000D3585560A025ED0050511BB2A14202D055
:1056A00015D2611ACB401800FEBD0823B6E71023BF
:1056B000B4E72023B2E74023B0E78023AEE701231D
:1056C000ACE708240026B1E70C000126AEE7091B71
:1056D0008B40E8E754B20000580000200070004002
:1056E000140000200405000018000020FF00FFFF48
:1056F000FC700040F0B51E285BD8364B8000C258C5
:10570000354B1E68002E30D1C227344BBF00D8590C
:10571000334C03250440C02000022043D851C0244C
:1057200080206400800018512E4F18602E4B803C62
:10573000D859FF3CA043D8510437D859A843204337
:10574000D8510837D8590C35A843844607206546F8
:105750002843D851A820C0001E50C12080268000B8
:1057600076021E501C601C4B1C60142500202B0070
:105770001E4C2E0046433659771C1BD14343E25042
:10578000A0230325C132FF329200DB05D550184B10
:105790001A68082A14D114234343E3189A6812485C
:1057A0005132FF32920059601150DA68C1239B00D8
:1057B000C250F0BD9642E1D001300328D9D1F8E7BC
:1057C000082A02D9083AD140E5E708239A1A9140FD
:1057D000E1E7C04654B20000FC11002000E100E007
:1057E000FF00FFFF04050000009000401C000020A7
:1057F0005C0000202149F0B54A6C2148002A14D0F1
:10580000A025A12600230124ED05F600C258571C4F
:1058100006D0C7187F68002F02D027009740AF51ED
:1058200014333C2BF2D100234B64A0230121DB0570
:1058300000260F009C4614234B43C3181A1F1268FE
:10584000104C0E4D920014195219526C002A10D0AF
:105850001A00143A1268551C09D0103B1B68FF2B24
:1058600005D03B00934065461A00074BEA50FC34D4
:10587000666401310429DED1F0BDC046FC900040D1
:105880001C000020009000400C05000000B51E2800
:1058900010D80C4A8000835803290BD8A022080096
:1058A000C133FF33D2059B0001F0FCFA0209050762
:1058B0000021D15000BD0C21FBE70421F9E70321B1
:1058C000F7E7C04654B200001E280AD8074B8000F4
:1058D000C25801239340A022D205002902D10449D5
:1058E00053507047A121C900FAE7C04654B20000E6
:1058F0000C050000030000201E2B0AD8A021A222C4
:10590000C905D2008858034A9B009B58D840012300
:105910001840704754B20000F7B506000D000C00A7
:105920008B180193019B671B9C4207D03368217839
:105930001B683000984701340028F3D13800FEBDC1
:105940000849094A094B10B51B688858FA22190AF8
:105950001B0618439200002301F070FC4904C00BA1
:10596000084310BD00100140040500000012002093
:1059700070B5041E09D0FFF7E3FF050000F014F82E
:10598000FFF7DEFF401BA042F8D370BD0022044B9E
:105990009A60044A13680133DBB213607047C04653
:1059A000FC1001400012002070470000F0B5C64610
:1059B00000B5CB0F9846404A4B005B0D9A1882B059
:1059C0000D000400132A2FDC002A49DB3B4F17414E
:1059D0003E000E40064323D07F08390029400C4387
:1059E0000AD03749BD438C4663445C425C41802306
:1059F000DB021341E4071D434146CE0031492B0031
:105A00008E192200346875682000290001F0BCFD61
:105A1000009001910098019922002B0002F04AFCAD
:105A200002B004BC9046F0BD332A08DD8023DB00C1
:105A30009A42F5D102000B0001F0A6FDF0E7224AE0
:105A40009446012263445242DA400242E8D05208AE
:105A50000242D1D094438022D2051A411443CBE7AD
:105A60004B005B080343DBD00B031B0B1C4363425F
:105A7000234380244D0C24031B0B23406D042B4334
:105A800019004346DA000F4B9B181C685D68020042
:105A90000B002000290001F077FD00900191009893
:105AA000019922002B0002F005FC42464B005B08E6
:105AB000D60733431900B3E701FCFFFFFFFF0F00D8
:105AC000EEFBFFFF00B30000EDFBFFFFF8B5274A38
:105AD0004B005B0D9A180C000700132A10DC002AFB
:105AE00036DB234B13410B423AD08024240314416C
:105AF000002064189C430600250030002900F8BDF2
:105B0000332A0EDD80230600DB000D009A42F4D11B
:105B100002000B003800210001F036FD06000D00E8
:105B2000EBE7144D0600AC46012563446D42DD40B1
:105B3000AC4663460D000342DFD033239A1A323B52
:105B400093401818874200D94C1C63469843D2E70B
:105B5000C90FCC070020531CCDD1074B1C43CAE70B
:105B600006000D000028C0D1C7E7C04601FCFFFFBA
:105B7000FFFF0F00EDFBFFFF0000F03F30B5214AB3
:105B80004B0087B05B0893421EDD1F4A934205DD40
:105B900002000B0002F08EFB07B030BD02AA00F03D
:105BA00035F803231840049A059B012813D00228D6
:105BB0001DD0002814D00298039900F037FA8023F2
:105BC0001B069C466144E7E7002300220093002364
:105BD00000F0A6FFE0E70298039900F027FADBE760
:105BE000012402980399009400F09AFFD4E701245D
:105BF00002980399009400F093FF80231B069C46B3
:105C00006144C9E7FB21E93FFFFFEF7FF0B54E4656
:105C10004546DE465746E0B5E14B4C008FB0904616
:105C2000894664089C4200DC87E0DE4B9C4222DC13
:105C3000DD4A002900DC92E0DC4B02F03BFBDB4B51
:105C400006000F009C4200D17EE1D94AD94B02F0F8
:105C500031FB02000B00414630000A604B60390006
:105C600002F028FBD34BD24A02F024FB4346012525
:105C70009860D9606BE0D04B9C4200DC8FE0CF4B4A
:105C80009C4200DD55E1CE4A231592469A44514686
:105C90000905631A19001D00040002F053FE02F00A
:105CA00087FE02000B00200029000892099302F0F1
:105CB00001FB0022C34B02F08BF80F00060002F03C
:105CC00041FE02F075FE04000D0002000B003000E2
:105CD00039000A940B9502F0EDFA0022B94B02F05C
:105CE00077F8002200230C900D9101F079FA00283A
:105CF00000D192E1002300222000290001F070FA77
:105D0000434243410133B04A41460192022208A86E
:105D10000092524600F0A4FA4B460500002B16DA1A
:105D2000802243461206944642465B6845426344DD
:105D30005360D3686344D36009E00B00020041461E
:105D40000A604B600022002300258A60CB60280097
:105D50000FB03CBC90469946A246AB46F0BD934B73
:105D600001F012FC914B06000F009C4200D13DE176
:105D70008F4A904B01F008FC02000B0041463000B6
:105D80000A604B60390002F095FA894A894B01F0AC
:105D9000FBFB012543466D429860D960D7E700F0D0
:105DA00071FF8A4A8A4B06000F0002F011F80022A8
:105DB000884B01F0E9FB02F0C5FD050002F0F8FD9B
:105DC000794A7A4B0490059102F002F802000B0028
:105DD0003000390002F06EFA754A06000F00049890
:105DE0000599744B01F0F4FF029003911F2D00DC24
:105DF000C7E0029A039B3000390002F05BFA834649
:105E00008A4653465B0024155B0DE31A102B6CDDAC
:105E100004980599D322674B520501F0D9FF02007F
:105E20000B00300039000292039302F043FA0A009B
:105E3000010013000691079202003900300002F0C1
:105E400039FA029A039B02F035FA06000F00049813
:105E50000599614A614B01F0BBFF32003B0002F043
:105E600029FA069E079F0B000200390030000292BB
:105E7000039302F01FFA4B005B0D83468A46E41A37
:105E8000312C32DD04980599B822544B920501F06B
:105E90009FFF03000C000200029303940B0006987E
:105EA000079902F007FA02000B0006000F0006989F
:105EB000079902F0FFF9029A039B02F0FBF9484AA6
:105EC0000290039104980599464B01F081FF029AD4
:105ED000039B02F0EFF902000B0030003900029240
:105EE000039302F0E7F983468A465A4653464146F1
:105EF00030000A604B60390002F0DCF9029A039B23
:105F000002F0D8F944460B000200A260E3604B4661
:105F1000002B00DB1BE75B46236080231B065344FA
:105F2000636080231B069C466144A060E1606D4273
:105F30000DE70B00020002F0BDF943460025986012
:105F4000D9601860596002E7D3221A4B520502F05B
:105F5000B1F9214A214B0D00040002F0ABF9020017
:105F60000B00414620000A604B60290002F0A2F9B4
:105F70001A4B194A02F09EF9434601259860D960F0
:105F8000E5E602000B003000390002F093F96B1EC9
:105F9000154A9B009B5883468A46A342A5D130E709
:105FA000FB21E93F7BD9024000004054FB21F93F2F
:105FB0003163621A61B4D03DFB213941FFFFEF7FAD
:105FC000EAFBFFFF0000704190B3000083C8C96D79
:105FD000305FE43F0000E03F7370032E8A19A33B5B
:105FE000C14920259A837B3910B30000D3220C4B82
:105FF000520501F0C9FA0B4A0B4B04000D0001F0E9
:10600000C3FA02000B00414620000A604B602900E1
:1060100002F050F9034A044BB9E6032373E6C04685
:1060200061B4D03D7370032E8A19A33BF0B5474687
:10603000CE4680B587B000920193754B4F008146E4
:1060400088467F089F4263DC02F07CFC002800D178
:10605000D4E04A4643464846414601F0B9FE0400B2
:106060000D006C4A6C4B01F0B3FE6C4A6C4B01F0B6
:106070008BFA22002B0001F0ABFE6A4A6A4B02F059
:1060800019F922002B0001F0A3FE684A684B01F0C9
:106090007BFA22002B0001F09BFE664A664B02F061
:1060A00009F922002B0001F093FE644A644B01F0D1
:1060B0006BFA22002B0001F08BFE0290039100226C
:1060C000604B2000290001F083FE029A039B06002A
:1060D0000F002000290001F07BFE009A019B0400C4
:1060E0000D004846414601F073FE02000B002000FF
:1060F000290002F0DFF802000B003000390002F046
:10610000D9F802000B0000204F4902F0D3F870E0EC
:1061100002000B0001F05CFE04000D003D4A3E4B06
:1061200001F056FE3D4A3E4B01F02EFA22002B00B4
:1061300001F04EFE3B4A3C4B02F0BCF822002B0023
:1061400001F046FE394A3A4B01F01EFA22002B00BC
:1061500001F03EFE374A384B02F0ACF822002B002B
:1061600001F036FE354A364B01F00EFA2B002200C4
:1061700001F02EFE354B029003919F429FDD344B80
:1061800000229F423DDC334900207B182E49160037
:106190001F0002F08FF8049005910022294B200087
:1061A000290001F015FE32003B0002F083F8029A4C
:1061B000039B06000F002000290001F009FE009A51
:1061C000019B04000D004846414601F001FE02001B
:1061D0000B002000290002F06DF802000B003000D7
:1061E000390002F067F802000B000498059902F0EC
:1061F00061F807B00CBC90469946F0BD00201249EA
:10620000F7E7154B002604920593144FC5E7C046E7
:10621000FFFF3F3ED43888BEE9FAA8BDC4B1B4BD83
:106220009EEE213EAD529C804F7E923E9015CB1942
:10623000A001FA3E7751C1166CC1563F4C555555D9
:106240005555A53F0000E03F0000F03F3233D33FFB
:106250000000E93F0000E0FF0000E73F0000D23F00
:10626000F0B5DE464E4645465746E0B5DC4CA54403
:106270000D9114001900A49A0993DA4B9200D65894
:106280004D1E03901821E01E0696029500F09EFE1A
:10629000C3430100DB1719404B1C9A009B1ADB001B
:1062A0001B190B9105934C1B771918D4A59BA500BE
:1062B0009C463F1922AE6544013707E0286802F08A
:1062C00077FB013403C60435BC4208D0002CF5DA54
:1062D00000200021013403C60435BC42F6D1069BE0
:1062E000002B01DA00F0FDFB069B03990133DB0074
:1062F0009A46099BDA00944600920022914672AABF
:106300000492B94A6144934688469AAB63449B44DD
:10631000029B002B00DABCE15D4600260027039CAF
:106320004D442A686B6803CC01F052FD02000B005B
:106330003000390001F028F9083D06000F004445FF
:10634000EFD1049B4B441E605F6008239C46E144F0
:10635000D145DDD10EA804218446494261448C46D2
:10636000069A93009C44614684460A910399083B2F
:1063700063448C460C93009B009263449B46009AB6
:106380000498D10003008C46634408911E685F683E
:10639000002A33DD954980468C466244D3009844F8
:1063A00070AB9A460EAB99460022914B30003900F3
:1063B00001F00EFD02F0C6FA02F0FAFA00228D4B4F
:1063C00004000D0001F004FD02000B003000390054
:1063D00001F070FF02F0B6FA4B4601C399464346FE
:1063E00020001A685B68290001F0CEF808235B42A0
:1063F0009C46E04406000F00D045D5D1059B3000F7
:106400001A003900984600F0DDFCFF2300229B05AE
:1064100004000D0001F0DCFC00F038FC0022764B9B
:1064200001F0D6FC02000B002000290001F042FF21
:106430000D00040002F086FA814602F0B9FA02006B
:106440000B002000290001F035FF060040460F0038
:10645000002800DCEEE0009B18215A1E92000EABD3
:106460009B58091A1D000D41A9448D405D1B0EABC0
:106470009D5017231B1A1D41002D2DDD01239C4625
:10648000009BE144002B00DC1CE20E9C0123002C4D
:1064900000D0B5E0009A012A09D099000EAA5458FC
:1064A0000133002C00D0ACE0009A9A42F5D1059B54
:1064B000002B0EDD012B00D1A8E1022B09D1009B9E
:1064C0000EA95A1E92000EAB9B5807939B029B0A83
:1064D0008B50022D00D1C1E0002300223000390092
:1064E00000F07EFE009B002800D194E2069A591E1F
:1064F0008A4210DC414A0A9894460EAA63449446A4
:1065000000229B0063441C68043B22438342FAD16F
:10651000002A00D0C0E0069B0EAA013B9B00D35886
:10652000002B00D0B3E001220C9B043B59680132E0
:106530000029FAD0009B9C466244110007921A0081
:1065400001338B4246DC0B9863468046A59C43444E
:10655000A046099C9B00A1464A449844D30022AA25
:106560009146049A99449446089BA59A63448446AC
:10657000614494469A468B006344009343465868AE
:1065800002F016FA4B4618605960029B002B24DB80
:106590004D46039C0026002701E0286869680CCC62
:1065A00001F016FC02000B003000390000F0ECFF97
:1065B000083D06000F005C45EFD153469E60DF604A
:1065C00004239C460433E0449C46009BE144E2449F
:1065D0009845D3D1079B0093D1E600260027ECE72E
:1065E00094FDFFFFD8B4000018FEFFFFFFFFFF1F60
:1065F0000000703E0000704100002040FFFFFF3FA0
:10660000002180225204141B0EAA54500099994272
:106610000EDD0EA884469B000EAA8900D258614464
:106620006344CF4800E01A68821A04C38B42FAD14F
:1066300001243CE7059B002B06D1009B0EAA013BE1
:106640009B00D558ED1517E70022C64B300000F02F
:10665000EBFD002800D024E100253DE732003B009F
:106660000020C14901F026FE06000F00002C00D1D9
:1066700032E7059A0020BC4900F0A4FB02000B00A1
:106680003000390001F016FE06000F0024E7012259
:1066900050E70026002754E64B46059A07938846A4
:1066A0008B000EA9CB58183A08950592002B0DD1F6
:1066B0008C464146AD4B43449B006344043B5868C1
:1066C0000139183A0028F9D088460592059A002029
:1066D000A54900F077FB434604000D00002B00DACB
:1066E00005E29E000EAB9C464346DB0066449C469A
:1066F000059370AB9946049F67440097306802F099
:1067000057F922002B0001F063FB0022386079600A
:10671000974B2000290001F05BFB083F04000D00AF
:10672000043EB945EAD14AAB03939B4600239A46FF
:10673000069B4246994643460132029204934B46D9
:10674000002B00DAAAE080208A4B009D9846C00505
:10675000894900260027002408E008239C460835C4
:10676000E044544511DC4346186859682A686B6850
:1067700001F02EFB02000B003000390000F004FF96
:10678000013406000F00A145E7DA5B46C0C39B4613
:1067900001239C46009BE244083B0093029B9A45E0
:1067A000CDD1049B9846A49B022B00DD8EE0002BEC
:1067B00037DC1FD1059B00271D00039B00249C464E
:1067C0001E006544083E2A686B683800210000F00E
:1067D000DBFE083D07000C00AE42F4D1089B002B05
:1067E00003D080231B069C4664443A0023000D9985
:1067F0000A604B600720079B18409B239B009D4429
:106800003CBC90469946A246AB46F0BD009B0EA903
:106810005A1E92000EAB9B5807935B025B0A8B508B
:1068200057E64346002B00DA70E100200021DB0030
:106830004AAAD61848AF32687368083E00F0A4FE32
:10684000B742F8D1089B002B00D025E10B000200D5
:106850004A984B990D9C2260636001F02BFD4346E2
:1068600007000C00002B13DD01254CAEB1463800AB
:106870002E0021004C4601360CCC00F085FEA146CE
:10688000B045F7DA089B07000C00002B00D015E19B
:106890003A0023000D998A60CB60ABE70026002701
:1068A00073E701239C46009BE1440225002B00DD99
:1068B000EBE532003B0000202B4901F0FBFC060019
:1068C0000F0009E60024F2E54AAB0393A49B032BD7
:1068D00000D08FE74346002B00DC14E1039ADB0075
:1068E0009B46130091465B441E685F68234B4344FC
:1068F0000293DB00994448AB9A464B465C681B68A0
:106900001800210032003B000090019100F03CFE95
:1069100004000D0002000B000098019901F0CAFC70
:106920003B00320000F030FE4B469860D9601C609E
:106930005D6008235B429C46E14426002F00CA4567
:10694000DBD14346012B00DCE3E0039A13005B44F8
:106950001E685F68029BDB0099464A44904610E03F
:10696000FFFFFF000000E03F0000F03FFFFFFF3FA0
:106970000000703E98B40000FB21F93FFFFFFF1FAD
:10698000984643465C681B681800210032003B00B3
:106990000090019100F0F8FD04000D0002000B00D2
:1069A0000098019901F086FC32003B0000F0ECFDFC
:1069B0004346039A9860D9601C605D60083B2600DE
:1069C0002F009A42DCD14D469446002600244746CB
:1069D000083565442A686B683000210000F0D4FD5A
:1069E000083D06000C00AF42F4D1039B4A9F5D684E
:1069F0009968D868089B002B65D0802212069446BF
:106A00000D9B6544604464441F605D609960D8607C
:106A10001E615C61EEE69A464B460793059B30008B
:106A20005A423900089500F0CDF900223A4B060091
:106A30000F0000F0F9FB002824D0384B0022300072
:106A4000390001F0C5F901F07DFF524604009500C0
:106A500001F0AEFF0022304B01F0BAF902000B004A
:106A60003000390001F026FC01F06CFF0EAA5051F5
:106A70000122059B524418339046059393000EAAB9
:106A8000D45023E65346300039009C0001F05AFFF1
:106A90000EAB1851D04619E680230D9A1B06CB1871
:106AA000106053600B0002004A984B9901F002FC01
:106AB000434607000C00002B00DDD5E680231B06B3
:106AC0009C466444E4E62B003A000D9D2A606B600E
:106AD0000A000300AA60EB60320023002A616B61A8
:106AE00088E6099BDB00009372AB049332E4A49B1D
:106AF000022B00DDE8E6002B00DD92E600D079E60F
:106B0000002700246AE6002600246EE7002000210A
:106B100098E60026340068E7000070410000703EEF
:106B2000F0B5CE46474680B587B000920193474AFC
:106B30004B00814688465B08934207DC4146484645
:106B400001F000FF4146031E484666D04A464346D0
:106B50004846414601F03CF904000D0002000B00DC
:106B60004846414601F034F9394A3A4B06000F00D5
:106B70002000290001F02CF9374A384B01F09AFB2C
:106B800022002B0001F024F9354A364B00F0FCFCC2
:106B900022002B0001F01CF9334A344B01F08AFB30
:106BA00022002B0001F014F9314B324A00F0ECFCCA
:106BB0000E9B02900391002B34D000980199002283
:106BC0002D4B01F005F9029A039B049005913000CA
:106BD000390001F0FDF802000B000498059901F05E
:106BE00069FB22002B0001F0F3F8009A019B01F0F1
:106BF00061FB224A04000D00214B3000390001F0F6
:106C0000E7F802000B002000290000F0BDFC0200A4
:106C10000B004846414601F04DFB07B00CBC9046C6
:106C20009946F0BD02000B002000290001F0D0F8C9
:106C3000124A134B01F03EFB32003B0001F0C8F852
:106C40004A46434600F0A0FCE7E7C046FFFF3F3E50
:106C50007CD5CF5A3AD9E53DEB9C2B8AE6E55A3EE6
:106C60007DFEB157E31DC73ED561C119A0012A3F82
:106C70001111813FA6F810110000E03F495555550C
:106C80005555C53F49004B0819007047474AF0B5B4
:106C90004F4691464B005B0D99444646D6464A46C0
:106CA000C0B505000C000E0088460700132A27DC3B
:106CB000002A4BDB3E4B13419A460B0052461340D1
:106CC000034318D03B4A3C4B2800210000F05CFCF9
:106CD0000022002300F09EFA002847D0002C04DA9E
:106CE00080234A465B031341984446465346002797
:106CF0009E43380031001CBC90469946A246F0BD28
:106D0000332A08DD8023DB009945F4D102000B0013
:106D100000F03AFCEFE7294A9446012263445242CC
:106D2000DA4092460242E6D0224A234B2800210054
:106D300000F02AFC0022002300F06CFA002815D095
:106D4000002C1EDB534646469F430FE0194A1A4B60
:106D50002800210000F018FC0022002300F05AFA5D
:106D6000002803D0002C04DB002700263800310067
:106D7000C1E76400640825430027002DF6D0104EBB
:106D8000F4E74B46142B0BD03422D21A0123934044
:106D90005D19BD4208D201239C462F00E044D1E793
:106DA000133B9C46E044CDE72F00CBE701FCFFFFFF
:106DB000FFFF0F009C7500883CE4377EEDFBFFFF72
:106DC0000000F0BF4B0070B55B0D14000A00002BF3
:106DD0001AD14B005B08034315D0234B002200F06F
:106DE000F7FF224B9C422DDB0A004B005B0D363B2C
:106DF0001F4DE318AB422ADC002B0DDD1D4C1B059B
:106E000022401A43110070BD1B4DAB42F0D102006D
:106E10000B0000F0B9FBF6E71D00353519DA174B0A
:106E200002009C4209DD0B001548164900F032F8BB
:106E3000134A144B00F0CCFFE5E70B00124813494E
:106E400000F028F8104A114B00F0C2FFDBE7020007
:106E5000E9E7084C363322401B0513431900002292
:106E60000B4B00F0B5FFCEE700005043B03CFFFFF6
:106E7000FE070000FFFF0F80FF07000050C3000067
:106E80009C7500883CE4377E59F3F8C21F6EA5015B
:106E90000000903C30B54A00DB0FDB0752081A4374
:106EA000110030BD02B4714649084900095C49002F
:106EB0008E4402BC7047C046002243088B4274D304
:106EC00003098B425FD3030A8B4244D3030B8B42EB
:106ED00028D3030C8B420DD3FF22090212BA030CF4
:106EE0008B4202D31212090265D0030B8B4219D3D5
:106EF00000E0090AC30B8B4201D3CB03C01A5241F5
:106F0000830B8B4201D38B03C01A5241430B8B423C
:106F100001D34B03C01A5241030B8B4201D30B0325
:106F2000C01A5241C30A8B4201D3CB02C01A52414C
:106F3000830A8B4201D38B02C01A5241430A8B420F
:106F400001D34B02C01A5241030A8B4201D30B02F8
:106F5000C01A5241CDD2C3098B4201D3CB01C01A12
:106F6000524183098B4201D38B01C01A524143091C
:106F70008B4201D34B01C01A524103098B4201D30A
:106F80000B01C01A5241C3088B4201D3CB00C01A77
:106F9000524183088B4201D38B00C01A52414308EF
:106FA0008B4201D34B00C01A5241411A00D2014614
:106FB000524110467047FFE701B5002000F0F0F89D
:106FC00002BDC0460029F7D076E7704703460B4361
:106FD0007FD4002243088B4274D303098B425FD3D2
:106FE000030A8B4244D3030B8B4228D3030C8B42FE
:106FF0000DD3FF22090212BA030C8B4202D31212E4
:10700000090265D0030B8B4219D300E0090AC30BB8
:107010008B4201D3CB03C01A5241830B8B4201D365
:107020008B03C01A5241430B8B4201D34B03C01A4E
:107030005241030B8B4201D30B03C01A5241C30AC6
:107040008B4201D3CB02C01A5241830A8B4201D337
:107050008B02C01A5241430A8B4201D34B02C01A21
:107060005241030A8B4201D30B02C01A5241CDD2C6
:10707000C3098B4201D3CB01C01A524183098B4211
:1070800001D38B01C01A524143098B4201D34B01FA
:10709000C01A524103098B4201D30B01C01A52415D
:1070A000C3088B4201D3CB00C01A524183088B42E4
:1070B00001D38B00C01A524143088B4201D34B00CD
:1070C000C01A5241411A00D201465241104670473F
:1070D0005DE0CA0F00D04942031000D34042534044
:1070E00000229C4603098B422DD3030A8B4212D304
:1070F000FC22890112BA030A8B420CD38901921136
:107100008B4208D3890192118B4204D389013AD072
:10711000921100E08909C3098B4201D3CB01C01A47
:10712000524183098B4201D38B01C01A524143095A
:107130008B4201D34B01C01A524103098B4201D348
:107140000B01C01A5241C3088B4201D3CB00C01AB5
:10715000524183088B4201D38B00C01A5241D9D2CD
:1071600043088B4201D34B00C01A5241411A00D24E
:107170000146634652415B10104601D34042002B4A
:1071800000D54942704763465B1000D3404201B5C9
:10719000002000F005F802BD0029F8D016E770477E
:1071A0007047C046D0400B1C1141203A03D49C4686
:1071B0001341184363465242934018437047C046F8
:1071C0008446101C62468C46191C634600E0C0468B
:1071D0001FB500F095FD002801D40021C8421FBD55
:1071E00010B500F0EDFC4042013010BD10B500F0CC
:1071F00087FD002801DB002010BD012010BDC04626
:1072000010B500F07DFD002801DD002010BD01203B
:1072100010BDC04610B500F00FFD002801DC0020B5
:1072200010BD012010BDC04610B500F005FD0028BE
:1072300001DA002010BD012010BDC046F0B5CE46D9
:10724000474615042D0C2E0080B50704140C3F0C86
:107250009946030C7E435D43674363437F19340CB7
:10726000E4199C46A54203D980235B029846C44496
:107270004B4643435143250C36046544360C2404E5
:10728000A4195B19591820000CBC90469946F0BD12
:10729000F0B54E4657464546DE46E0B543025B0A2A
:1072A000450083B00F1C99462D0EC60F002D57D0F8
:1072B000FF2D24D08020DB00C0041843002381462A
:1072C0009A469B467F3D7C027A00FB0F640A120EB1
:1072D000984623D0FF2A4BD0E30080240020E4040A
:1072E0007F3A1C43AD186B1C4746019353467740C9
:1072F0003A000F2B48D87D499B00CB589F46002B66
:1073000000D085E008339A46063B9B467C027A0013
:10731000FB0FFF25640A120E9846DBD1002C00D02B
:1073200090E0524601231A4392460120DBE74C4687
:1073300058461700022824D0032800D1CFE00022AD
:10734000002301284DD15802D205400AFF071043FF
:10735000384303B03CBC90469946A246AB46F0BDCC
:10736000002B5BD104239A46033B00259B46AAE7EA
:10737000FF35002C60D1524602231A439246022068
:10738000B1E7FF220023DEE74B461B0C9C464B4631
:107390002604360C180461463300220C6446000CA7
:1073A00043434E435043544380191A0C12189642DB
:1073B00003D9802149028C4664441B041B0C100431
:1073C000C01883015E1EB341800E1843130C1B19B5
:1073D0009B0103431C00230179D5012362081C4053
:1073E0001443019A7F32002A4DDD630704D00F2336
:1073F0002340042B00D00434230103D53C4B019AD5
:107400001C408032FE2ABCDCA3015B0AD2B29AE7A0
:107410000C239A46093BFF259B4654E7180001F0D0
:1074200053FB4A46431F76259A4000236D429146FE
:107430002D1A9A469B4646E7524603231A43924624
:10744000032050E7200001F03FFB431F2D1A9C4012
:10745000763D002047E780230027DB03FF2272E709
:10746000424666E74C463200584662E780234A4669
:10747000DB031A4222D01C4220D123435B025B0A69
:107480004746FF225FE701239A1A1B2A21DC2300CB
:107490000199D3409E318C401A0023005C1EA34109
:1074A00013435A0704D00F221A40042A00D0043391
:1074B0005A0111D49B015B0A002244E780234A460B
:1074C000DB0313435B025B0A3700FF223BE70195B6
:1074D00087E70022002336E70122002333E78023D9
:1074E000DB0323435B025B0AFF222CE7E8B40000C6
:1074F000FFFFFFF770B500283DD0C317C5185D40EA
:10750000C40F280001F0E0FA9E22121A962A07DC26
:10751000D2B2082833DD083885406802400A23E0EB
:10752000992A0BDD052329001B1AD94003001B33C0
:107530009D402B005D1EAB4119430D00052801DD68
:10754000431F9D402B000F490B406E0709D00F26AB
:107550003540042D05D004335D0102D59F220B4038
:10756000121A9B01580AD2B24002D205400AE4071F
:107570001043204370BD002400220020F4E768027D
:10758000400AF1E7FFFFFFFBF0B54F464646D646FF
:107590000C000903C0B5490A470F5E0039431F03B9
:1075A000DB0F9C4665007B0A570F1F436D0DE40FF0
:1075B000760DA146C000B846D200AB1B64457BD017
:1075C000002B5FDD002E00D0A4E03E00164300D16A
:1075D00012E15E1E002E00D09EE1871A4346B8429B
:1075E00080410125C91A4042091A0B0200D431E139
:1075F00049024E0A002E00D16EE1300001F064FA1B
:107600000300083B1F2B00DD61E120223900D21A64
:107610009E40D1409F400E439D4200DD51E15D1BE5
:107620006B1C1F2B00DD7CE12021C91A3D003000BE
:107630008F408840DD40791E8F413100072228436A
:10764000D940002507433A40002A09D00F233B4088
:10765000042B05D03B1DBB42BF417F42C9191F000F
:107660000B0200D426E26A1CC64B55056D0D9A42EA
:1076700000D106E1C44AFF080A40530752023B43C7
:10768000120B8EE0002B00D0B8E06B1C5B055B0D8D
:10769000012B00DC30E1871A4346B842B641CB1AD1
:1076A00076429E1B330200D54CE13B003343A1D10F
:1076B00000220024002570E0002B00DCE5E0002E15
:1076C00000D183E0AF4EB54260D080263604374308
:1076D000B846382B00DC3EE1434613431F007A1EB8
:1076E00097413F1887428041404209180B0200D45D
:1076F000B0E0A44B01359D4200D1C3E0A24A7B0813
:107700000A4001210F401F435108D30707221F439E
:107710003A4099E79B4EB54238D08026360437432D
:10772000B846382B00DDDCE01F2B00DC30E11E000A
:107730004746203EF740BC46202B04D04026F31A93
:1077400046469E403243170063467A1E97411F43C8
:10775000CCE0002B00D104E24346134300D159E1B1
:107760004B07C00818438023C9081B03194208D0DF
:107770004546ED081D4204D14346D0085907084349
:107780002900420FC9007F4D1143C0004B07CA08B2
:107790007C49C00803438D4268D012036D05120B6B
:1077A0006D0D002112031800130B0A0D12051A4368
:1077B000764B2D0513402B435B00E4075B08234306
:1077C00019001CBC90469946A246F0BD3E001643E7
:1077D00012D05E1E002E00D000E187188742804143
:1077E00041444042091801250B0233D5022585E7A3
:1077F00064463300414610001D00C7E7002D00D04D
:10780000DAE00C000443F3D05C1C00D19FE15D4C36
:10781000A64200D12FE1DB43382B00DD66E11F2BB0
:1078200000DD83E120240500E41A0F00DD40D9408B
:10783000A0404346A7405B1A441EA04198462F43F0
:107840003843171ABA42924143465242991A644643
:107850003500CAE607223A40002A00D0F6E64B0778
:10786000CA084849FF083B438D4296D1190011438D
:1078700000D19EE1802109030A431203120B414DFE
:107880008FE71500002200238BE7002B00D0C7E014
:107890006B1C5F057F0D012F00DCF1E0394DAB4221
:1078A00000D1B9E085180A00854289414244494225
:1078B00051180722CF076D082F4349083A401D0091
:1078C000C2E607223049ED1A31403A40BCE63E009C
:1078D0002838864000279FE6380001F0F5F8203070
:1078E0008EE6434613431F007A1E9741C71BB842DA
:1078F00080414042091A78E60E003B0006431343DC
:10790000002D61D1002E00D0F4E0002B00D11BE14E
:1079100064463900100039E71A4FBB427AD0330071
:10792000FFE630001F3DE840202B03D04021CB1A5A
:107930009E4037437B1E9F41072207433A40002168
:10794000002589E7171A4346BA42B641591A7642CA
:107950008E1B64464EE61F2B00DDADE02026474619
:10796000F61AB740B9461700B246DF404E463E43CE
:1079700037005646B240561EB24117434246DA40DF
:107980008918AEE6FF070000FFFF7FFFFFFF0F80B3
:1079900020264746F61AB740B9461700B246DF40E0
:1079A0004E463E4337005646B240561EB24117433C
:1079B0004246DA40891A99E77F4CA6425BD0802480
:1079C00024045B42214327E7002E0CD1002B00D179
:1079D000CBE0644639001000774DD7E6764FBB42C6
:1079E00018D0330075E6002B14D04B07C00818439D
:1079F0008023C9081B03194207D0FC081C4204D18C
:107A00007907D0080843E14621004C46420FC900DF
:107A10001143C000684DB9E61D0000220023C0E6F6
:107A2000002D5BD10D00054300D1E2E65D1C00D1C5
:107A3000B0E0614DAE421FD0DB43382B71DC1F2B11
:107A400000DD96E020250F00ED1AAF40B946070093
:107A5000AA46DF404D463D432F005546A840D94039
:107A6000451EA84188440743BF189742924151429E
:107A7000414435003AE6644635004146100085E64B
:107A80000B000343002D00D063E6002BF5D04346E6
:107A9000134300D17AE68718874280410722414488
:107AA000404209183A400B0200D4D5E6434B013559
:107AB0001940C9E5380069E61E004746203EF740F8
:107AC000BC46202B04D04026F31A46469E40324343
:107AD000170063467A1E97411F4302E6364DAE42B9
:107AE000CAD080252D045B422943A6E70843411EE6
:107AF0008841A6E6002B00D148E6871A4346B842E3
:107B0000B641CB1A76429E1B33024BD5171A434619
:107B1000BA429241591A5242891A072264463A409F
:107B200092E501430F00791E8F419DE71C000F0075
:107B3000203CE740202B03D04024E31A994008431F
:107B4000411E884138437CE60022002425E6171AAE
:107B50004346BA429241591A5242891A6446350044
:107B600043E541461000144D10E680220024120324
:107B700080E61D000F00203DEF40BC46202B03D0C7
:107B80004025EB1A9940084307006346781E874159
:107B90001F4369E7871897429B4141445B42C918DC
:107BA0003500A3E53B003343CED0072231003A40F5
:107BB00052E600231A00F4E5FF070000FFFF7FFFF5
:107BC000F0B54F464646D6468446C0B58046194E67
:107BD00018030F034D00000B5C0082463F0B6D0D38
:107BE000C90F9146640DDB0F0120B5420AD0B442A3
:107BF00003D0A54201D157450CD01CBC90469946F4
:107C0000A246F0BD66463E43F7D1AC42F5D154469C
:107C10001443F2D10120C845EFD1994207D0002D7D
:107C2000EBD163461F433800471EB841E5E700200B
:107C3000E3E7C046FF070000F0B54F464646D6468C
:107C40004D00C0B50E03C90F8A462C491F035C00C6
:107C50008046360B6D0D91463F0B640DDB0F8D4258
:107C60001ED08C4216D0002D1ED130438446002CED
:107C700001D13A4323D06246002A1AD09A4529D02E
:107C8000514602200139084001381CBC90469946F3
:107C9000A246F0BD39001143E5D002204042F4E78E
:107CA0003043FAD1AC420FD0002C0FD13A43E7D089
:107CB0000CE00122013B934318000130E5E76346E5
:107CC0000020002BE1D0DBE73A43E6D19A45D7D13B
:107CD000A542D5DCA54205DBBE42D1D808D00020A4
:107CE000BE42D2D250460123013898430130CCE73E
:107CF000C845C5D80020C845F4D3C6E7FF07000033
:107D0000F0B54F464646D6464D00C0B50E03C90FE6
:107D10008A462E491F035C008046360B6D0D914646
:107D20003F0B640DDB0F8D4218D08C4211D0002D1B
:107D300018D130438446002C1ED13A431CD16346EF
:107D40000020002B30D05146022001390840013874
:107D50002AE039001143EAD0022025E03043FBD16C
:107D6000AC4226D0002C26D13A4324D151460220E1
:107D700001390840013817E06246002A0FD09A45C1
:107D8000E1D1A54205DBBE42DDD819D00020BE42BC
:107D90000AD25046012301389843013004E0012201
:107DA000013B9343180001301CBC90469946A24603
:107DB000F0BD3A43D0D19A45C5D1A542C3DCE0E736
:107DC000C845C0D80020C845E3D3EDE7FF07000051
:107DD000F0B55746DE464E464546E0B583460600BA
:107DE0000F03480087B092461D003F0B400DCC0F9B
:107DF000002800D16FE0DE4B984238D08023FF008E
:107E00001B041F43730F3B430193DA4B0027994632
:107E100000239B46F60081442B0369001B0B52464E
:107E20009846490DED0F002900D185E0D04B9942CD
:107E300000D173E04346DA0080231B04134352460B
:107E4000CC48520F84461343524600206144D2006E
:107E500089442100694000918C46012149448A46A9
:107E60000F2F00D990E0C449BF00CF59BF465B46F1
:107E70003B43019300D06AE1022308270026814694
:107E80009B46C9E732005846019B61460091022893
:107E900000D175E0032800D1FEE1012800D02CE1DB
:107EA00000230027002600253F032A0D3F0BB3487F
:107EB00012053A4302401B051343009A5B00D107A9
:107EC0005B080B433000190007B03CBC9046994654
:107ED000A246AB46F0BD5B463B43019300D12FE188
:107EE000002F00D1A5E1380000F0EEFD03000B3BB0
:107EF0001C2B00DD96E11D22D31A5A460100DA4000
:107F00005E4608398F4013008E403B4301939C4BE3
:107F100000271B1A994600239B467DE7414653469E
:107F20000B4393498C46E144002B00D01AE1022216
:107F30000220174300228CE7134300D10DE1434692
:107F4000002B00D181E1404600F0BEFD02000B3A5B
:107F50001C2A00DD72E10100434608398B40984637
:107F60001D239A1A5346D3401A00434613435246E0
:107F70008A404946081A824989468144002068E7B8
:107F80007B4B002700268EE7140C1204120C110004
:107F9000370C3604350C794328008C462E0060439C
:107FA0006044834656432100300C8046584679434E
:107FB00040440291844506D98846802149028C4676
:107FC000E044414602913604010C360C00048B4615
:107FD00081191E0C1B041B0C0391190079438C465C
:107FE000280075436544A8465843050C454477432B
:107FF000A94203D9802149028C466744290C8C464A
:1080000039000004000C2D042D186144AB44059187
:108010005946049101990F043F0C080C3900514353
:108020004243904602008C46090C8B4662437C43D7
:1080300044445C44A04503D9802149028846424417
:10804000210C884661460904090C8C4639005943C5
:10805000434370437E430F0CF6182404BE19644456
:1080600042448C46B34203D980235B029846404485
:10807000029B61469846049B370443449B46AB45AC
:10808000AD416B420D0405992D0C8C467F19674458
:10809000FD18A8465D462D19A542A44193466442A9
:1080A000A446C344DC448F42BF4198459B4193455D
:1080B0009241A445A4415B427F421F43360C524289
:1080C0006442BF192243BF18624638184302D20DDA
:1080D000039913436A020A43501E82416146ED0D23
:1080E0002A434E023243D90100D4B3E0012650089E
:1080F00032400243DE0732435B08224C5444002CDA
:1081000062DD510709D00F201040042805D0101D52
:108110009042924152429B180200D90104D580241A
:108120001948E400034054441848844200DD27E71E
:108130005E075B02D2081F0B630516435B0DB2E6B8
:10814000002399460133042700269B4664E6032357
:10815000019781460C279B465EE6012201201743CA
:10816000002276E6032303201F43434671E6C04600
:10817000FF07000001FCFFFF28B50000FFFF0F8094
:108180000DFCFFFFFF030000FFFFFFFEFE070000E6
:108190000023802700933F030026434B83E6019B87
:1081A0003200A446584670E6AC466EE68027019938
:1081B0003F0339422DD03B422BD11F433F033F0B9E
:1081C00000951600384B6EE601252D1B382D00DD7D
:1081D00066E61F2D40DC35481C00504416008240E6
:1081E0008440EE40501E824134431443EB4062070A
:1081F00009D00F222240042A05D02200141D9442E7
:10820000804140421B181A023ED501230027002658
:1082100049E68027019B3F031F433F033F0B009428
:10822000214B40E603005A46283B9A400026019223
:108230006DE6584600F048FC203057E603005246F1
:10824000283B9A401300002293E6504600F03CFC85
:1082500020307BE6CA4650E71F201E004042041B28
:10826000E640202D03D0124C5444A3401A43501E24
:108270008241324307260027164009D00F200023F1
:10828000104014000428B9D122005E075B021F0BC6
:10829000D2081643002306E680273F031F433F030F
:1082A0003F0B1600004BFEE5FF0700001E04000018
:1082B0003E040000F8B557464E464546DE460C00E3
:1082C0000903E0B5490A460F5F0031431E03DB0F87
:1082D000760A9B46530F3343C84E6500C000E40F37
:1082E000D2006D0DA24681467F0D9C469046B74256
:1082F00000D1B9E05B46012673409B46EE1BA345C7
:1083000000D183E0002E63DD002F00D0B1E0634692
:10831000134300D123E1731E002B00D0BAE1861A6B
:108320006346B04280410125C91A4042091A0B0236
:1083300000D447E149024B0A98464346002B00D13E
:1083400089E1404600F0C0FB0300083B1F2B00DD25
:108350007CE120223000D21A4146D04099400200F0
:108360009E400A439D4200DD6AE15D1B6B1C1F2B92
:1083700000DD94E1202110003500C91A8E40DA405A
:108380008840DD40711E8E411100072228430025E0
:1083900006433240002A09D00F233340042B05D076
:1083A000331DB342B641764289191E000B0200D438
:1083B0003DE26A1C914B55056D0D9A4200D119E1C1
:1083C0008F4AF6080A40570752023743120B9BE0C8
:1083D000002E00D0C5E06E1C7605760D012E00DC67
:1083E00048E16746861ACB1BB042BF417F42B84680
:1083F0001F004346FF1A3B00B8461B0200D55FE151
:1084000037439AD100220024002579E0002E00DCB9
:10841000FAE0002F00D18DE0784B9D4267D0802399
:1084200067461B041F43BC46382E00DC52E16346FE
:1084300013435A1E93411E18864280414042091838
:108440000B0200D4BEE06D4B01359D4200D1D2E05D
:108450006B4A73080A4001210E401E435108D3079E
:1084600007221E43324095E71E00164300D045E721
:1084700040E7624B9D423AD0802367461B041F436E
:10848000BC46382E00DDEBE01F2E00DC3AE1330065
:108490006746203BDF403B00202E05D04027BF1B16
:1084A0006646BE40324390464646721E964133436E
:1084B000DAE0002B00D114E26346134300D168E1F7
:1084C00080234E07C008C9081B030643194208D081
:1084D0006046C008184204D163460100D2085E0716
:1084E0001643F3009946C900720F444D11434B46A1
:1084F000DE08424B4F073743CA089D4200D16EE069
:1085000012036D05120B6D0D00211203130B0A0DE2
:1085100012051A433B4B2D0513402B435B00E40728
:108520005B082343380019003CBC90469946A2469C
:10853000AB46F8BD6346134311D0731E002B00D029
:1085400007E18618864280416144404209180125AE
:108550000B0237D502257BE73E0061469146350088
:10856000C5E75C46002D00D0E1E00B000343F3D0EB
:10857000731C00D1ACE1214B9F4200D13AE1F3439F
:10858000382B00DD6FE11F2B00DD8CE120250E0074
:10859000ED1AAE40B0460600AA46DE4045463543D9
:1085A0002E005546D940A8406346451EA8415B1A97
:1085B0009C463043161AB242924163465242991A7F
:1085C0003D00B4E607223240002A00D0E4E60B4B1F
:1085D000F6084F073743CA089D4200D090E73B009A
:1085E000134300D1A6E180231B031A431203120B8D
:1085F000024D89E715000022002785E7FF070000EC
:10860000FFFF7FFFFFFF0F80002E00D0C7E06B1C35
:108610005E05760D012E00DCF0E0C84DAB4200D1C6
:10862000B9E085180A0085428941624449425118DF
:108630000722CE076D082E43490832401D00A9E6E7
:10864000BF49ED1A114007223240A3E63200283814
:108650008240002686E6300000F036FA203073E6CD
:10866000634613435A1E9341C61AB04280414042AA
:10867000091A5CE60E00674606431743002D5ED1DB
:10868000002E00D0F3E0002F00D11EE15C466146D1
:1086900091462CE7A94FBE427BD01E00F1E61000A8
:1086A0001F3DE840202B03D04021CB1A9A401643AF
:1086B000731E9E410722064332400021002583E7B6
:1086C000161A6346B2428041591A40420B1A984624
:1086D0005C4632E61F2E00DDABE02027BB1B9A462E
:1086E00063465746BB40994613004F46F3401F432D
:1086F0003B005746BA40571EBA4113436246F24008
:10870000891898E62027BB1B9A4663465746BB400C
:10871000994613004F46F3401F433B005746BA406B
:10872000571EBA4113436246F240891A9CE7834BB5
:108730009F425FD080252D047342294320E7002EFD
:108740000CD1002F00D1D0E05C46614691467B4DB4
:10875000CDE67A4FBE421CD01E0065E6002F18D031
:10876000C0084E0706438020C9080003014208D014
:108770006346DC08044204D12100DA46D2085E07D1
:108780001643F300994601245346C900720F114362
:108790001C406A4DABE61D0000220027B4E6002D08
:1087A00059D10B00034300D1D6E6731C00D1B2E0CF
:1087B000624B9F421ED0F343382B6FDC1F2B00DD32
:1087C00097E020250E00ED1AAE40B0460600AA46FE
:1087D000DE40454635432E005546A840D940451E4B
:1087E000A8418C440643B6189642924151426144D6
:1087F0003D0025E63D006146914678E60B000343C7
:10880000002D00D055E6002BF5D06346134300D170
:108810006DE6861886428041614440420918002274
:108820000B0200D4D0E6464B01351940B2E5B14603
:108830005DE633006746203BDF403B00202E05D03D
:108840004027BF1B6646BE40324390464646721ED6
:1088500096413343EFE5394B9F42CBD080252D0421
:1088600073422943A8E70843411E8841A2E6002F2E
:1088700000D13CE66346861ACF1AB0429B415B4268
:10888000FB1A98461B024ED5161A6346B242924115
:10889000591A5242891A5C4600227BE501430E00B8
:1088A000711E8E419FE71D000E00203DEE40B04638
:1088B000202B04D04025EB1A9940084381464846B6
:1088C0004346411E8841184374E60022002417E6FF
:1088D000161A6346B2429241591A5242891A3D0011
:1088E00025E561469146154D01E6802200241203DC
:1088F00079E61D000E00203DEE40B046202B04D04E
:108900004025EB1A9940084381464E464346711E66
:108910008E411E4367E7861896429B4161445B4245
:10892000C9183D008CE547463743CED00722414663
:10893000324049E600273A00E6E5C046FF0700005E
:10894000FFFF7FFF30B5144D0A034B00120B5B0D88
:10895000C90F0024AB4211DD104CA34210DC80246F
:10896000640322430E4CE41A1F2C0CDD0D48C31A7D
:10897000DA4013005C42002900D11C00200030BD09
:10898000094BCC18FAE7094DE040AC4663449A40E5
:1089900013000343EEE7C046FE0300001D04000081
:1089A0003304000013040000FFFFFF7FEDFBFFFF17
:1089B00070B500282DD0C317C5185D40C40F28001E
:1089C00000F082F8154B1B1A5B055B0D0A2815DDBC
:1089D0000B38854000222D032D0B002110002D03A4
:1089E0000A0D2D0B12052A430D4D1B052A4013437A
:1089F0005B00E4075B082343190070BD02002900F7
:108A0000153291400A000B21081AC5402D032D0B89
:108A1000E3E70024002300250022DEE71E04000017
:108A2000FFFF0F804100090E4B1C70B5DBB2460200
:108A3000750AC40F012B14DDE0239B006D07360B74
:108A4000CB1800210A0D280012051C4D32435B058E
:108A50002A405B0813435B00E4075B0823431900CB
:108A600070BD002914D1002D1ED0280000F02CF874
:108A70000A281CDC0B232A001B1ADA4003001533DA
:108A80009D400F4B12031B1A5B05160B5B0DD8E7BD
:108A9000002D06D0320B802636036D071643094B96
:108AA000CFE7084B0026CCE700230026C9E70300E8
:108AB0002A000B3B9A400025E3E7C046FFFF0F80EA
:108AC00089030000FF0700001C2101231B049842BA
:108AD00001D3000C10391B0A984201D3000A08394F
:108AE0001B09984201D30009043902A2105C401806
:108AF0007047C046040302020101010100000000AA
:108B00000000000030B51C00094B05001B6885B053
:108B1000D868084B002A01D1074B1A000292019332
:108B200000912B002200054900F020F800F01EFE05
:108B30006000002068B50000E6A4000075B50000E4
:108B4000084B10B50400002B02D0002100E000BF4C
:108B5000054B1868836A002B00D09847200001F06D
:108B600029FBC04600000000A4B500000EB403B508
:108B7000010003AB044804CB0068019300F020F926
:108B800002B008BC03B018476000002070B5002692
:108B90000C4D0D4C641BA410A64209D1002601F017
:108BA0000BFB0A4D0A4C641BA410A64205D170BDF4
:108BB000B300EB5898470136EEE7B300EB589847FF
:108BC0000136F2E73002002030020020300200209F
:108BD0004002002010B5034B0100186800F06AF84D
:108BE00010BDC0466000002010B5034B010018689E
:108BF00000F016F810BDC04660000020002310B53C
:108C00009A4200D110BDCC5CC4540133F8E7030094
:108C10001218934200D1704719700133F9E7000030
:108C200070B50500002910D00C1F2368002B00DA56
:108C3000E418280000F0CCFF1D4A1368002B05D172
:108C400063601460280000F0C4FF70BDA34209D91E
:108C5000216860188342F3D118685B68411821606D
:108C6000EEE713005A68002A01D0A242F9D9196828
:108C70005818A0420BD12068091858181960824270
:108C8000E0D110685268411819605A60DAE7A042D2
:108C900002D90C232B60D5E721686018824203D1EA
:108CA000106852684118216062605C60CAE7C04683
:108CB00004120020032370B5CD1C9D430835060027
:108CC0000C2D1ED20C25A9421DD8300000F080FFCB
:108CD000254A14682100002919D1244C2368002B4F
:108CE00003D1300000F04EFB20602900300000F07E
:108CF00049FB431C2BD10C233000336000F069FF8B
:108D000003E0002DDFDA0C233360002070BD0B6818
:108D10005B1B19D40B2B03D90B60CC18256003E027
:108D20004B688C420DD11360300000F052FF2000E0
:108D300007220B30231D9043C31AE7D05A42E2505A
:108D4000E4E763600C00EFE70C004968C3E7032326
:108D5000C41C9C43A042E1D0211A300000F012FB59
:108D6000431CDBD1C7E7C0460412002008120020D4
:108D7000936810B5013B9360002B04DA9469A34219
:108D800007DB0A2905D01368581C10601970080009
:108D900010BD00F01FFC0100F9E7F8B506000F0058
:108DA0001400D518AC4201D1002007E021783A0028
:108DB0003000FFF7DDFF0134431CF3D1F8BD0000A4
:108DC000F0B59FB002900F0016000593002805D063
:108DD00083690493002B01D100F0C8FD7B4B9F42B7
:108DE0005BD1029B5F68BB891B0762D53B69002B87
:108DF0005FD0002306AC6361203363761033A37623
:108E000035002B78002B01D0252B5CD1AB1B0493B4
:108E10000CD0320039000298FFF7BFFF431C00D18D
:108E2000C4E06269049B9446634463612B78002B21
:108E300000D1BBE0012200235242626002A95432F9
:108E400052186E1C2360E360A3601370A365317831
:108E500005225F4800F09EFE751C002835D122686F
:108E6000D30604D5532302A95B18202119701307D8
:108E700004D5532302A95B182B21197033782A2BB0
:108E80002CD0350000210A20E3682A786E1C303A85
:108E9000092A64D900292ED026E04E4B9F4202D1E8
:108EA000029B9F689FE74C4B9F429CD1029BDF68CF
:108EB00099E73900029800F0E3FB002899D00120DF
:108EC00040421FB0F0BD01359BE7414B2268C01AFC
:108ED00001238340134323602E00B8E7059B191D2F
:108EE0001B680591002B01DB099304E05B42E36002
:108EF0000223134323602B782E2B0AD16B782A2B65
:108F000035D1059B02351A1D1B680592002B2BDB02
:108F10000793324E29780322300000F03BFE0028F0
:108F200006D04023801B8340226801351343236011
:108F3000297806222A486E1C217600F02BFE002894
:108F40003AD0284B002B25D10722059B07339343AA
:108F5000083305936369039A9B18636150E74343A1
:108F600001219B18350090E701235B42D0E70023E5
:108F70000A201A000135636029786E1C30390929EE
:108F800003D9002BC5D00792C3E7424301235218EF
:108F90003500F1E705AB00933A00134B210002982E
:108FA00000E000BF0390039B0133D3D1BB895B0674
:108FB00000D584E70B9884E705AB00933A000A4B91
:108FC0002100029800F080F8ECE7C046FCB50000F4
:108FD000A8B500001CB60000DCB50000AEB500006E
:108FE000B2B50000000000009B8D0000F7B5150031
:108FF00001938A680B6900900C00934200DA130019
:1090000022002B6043321278002A01D001332B60FA
:1090100023689B0602D52B6802332B600627236842
:109020001F4027D0230043331B785A1E93412268E8
:10903000920630D42200019943320098089EB0472E
:10904000431C25D0062320682A68E16803400025D8
:10905000042B03D18D1AEB43DB171D40A368226953
:10906000934201DD9B1AED180027BD4220D100205C
:1090700010E00137E3682A689B1ABB42D2DD220068
:109080000123193201990098089EB047431CF0D182
:1090900001204042FEBD3020E1184331087021001C
:1090A0005A1C45310978A218433202331170C1E7C6
:1090B000220001231A3201990098089EB047431CF0
:1090C000E6D00137D1E70000F0B589B004920A007C
:1090D00043320593039002920A7E0C000E9B6E2A87
:1090E00000D186E01FD8632A33D008D8002A00D1E7
:1090F0008CE0582A4DD0250042352A7030E0642A91
:1091000001D0692AF7D1196825680A1D280629D5D2
:1091100008681A60002803DA2D23029A404213706F
:109120006B4E0A274FE0732A74D008D86F2A1FD0DD
:10913000702AE0D1202209680A43226003E0752AE0
:1091400016D0782AD7D12200782145321170614E8D
:1091500022E025001A684235111D196013682B7032
:10916000012365E008681A606906D3D500B2D1E72B
:1091700019682568081D186008682E0605D5544E24
:1091800008276F2A1BD00A2719E06D06F7D580B291
:10919000F5E745314E4E0A7018682268011D0068D7
:1091A0001960150621D5D30702D520231A43226062
:1091B0001027002803D1202322689A43226023002D
:1091C000002243331A706368A360002B58DB04222B
:1091D000216891432160002854D1029D002B5AD070
:1091E0002500337842352B7055E05506DBD580B22B
:1091F000D9E71A680D68101D4969186013682E06B2
:1092000001D5196002E06D06FBD519800023029D8F
:1092100023614FE01A68111D19601568002162680A
:10922000280000F0B7FC002801D0401B6060636894
:1092300023610023029A13703CE023692A000499F9
:109240000398059DA847431C3ED023689B0715D46F
:10925000079BE068984239DA180037E022000123C2
:10926000193204990398059EB047431C2CD0013550
:10927000E368079A9B1AAB42F0DCE9E70025F7E7C1
:109280000028ADD0029D3900FDF79CFE735C013DC6
:109290002B700028F7D1082F09D12368DB0706D5EA
:1092A00063682269934202DC3023013D2B70029BEC
:1092B0005B1B2361059B07AA00932100049B039875
:1092C000FFF794FE431CB8D10120404209B0F0BD25
:1092D000B9B50000CAB500000D4B70B51C6805009B
:1092E000A36B002B0FD11820FFF774FC094BA06370
:1092F0000360094B01224360084B83600B23838189
:109300000023026143610022A36B1D615A6170BD9D
:10931000600000200E33CDAB34126DE6ECDE0500AC
:10932000124B10B51C68A36B002B0FD11820FFF750
:1093300051FC0F4BA06303600E4B012243600E4BA8
:1093400083600B238381002302614361A46B0B4A7A
:10935000206961690A4BFDF771FF01220023801823
:109360005941206161614800400810BD6000002043
:109370000E33CDAB34126DE6ECDE05002D7F954C3F
:109380002DF45158002370B5064C050008002360E9
:1093900000F0FAFE431C03D12368002B00D02B60A1
:1093A00070BDC046BC2500200CB430B5164B9DB036
:1093B0000C1E1D6808DA8B2301202B6040421DB073
:1093C00030BC08BC02B01847822302A99B008B81E5
:1093D0000023029008619C4200D0631E8B604B61A9
:1093E00001235B42CB81209A21AB2800019300F03E
:1093F00079FC431C01DA8B232B60002CDFD0002387
:10940000029A1370DBE7C046600000200EB400B57E
:109410000B499CB01DAB029006900791049109483E
:10942000094904CB0591006802A9019300F05AFC98
:109430000023029A13701CB008BC03B01847C04642
:10944000FFFFFF7F600000200802FFFF02780B781B
:10945000002A03D0013001319A42F7D0D01A704768
:1094600003000A7801311A700133002AF9D17047DC
:109470000023C25C0133002AFBD1581E704730B56F
:109480000500002A00D130BD0C78013A6B1C2C700D
:109490000131002C05D19A189A42F4D01C70013386
:1094A000FAE71D00EDE70000F0B51F000E0087B0E1
:1094B0000590019102920C98347800F0EAFA0822A3
:1094C00000194378751C134036D12D2C36D1B51CAC
:1094D00074780126002F62D0102F09D1302C07D1CB
:1094E00020222B789343582B54D110276C780235C7
:1094F0002D4B3900F31818000393FDF763FD049119
:1095000001210023494202008C4618002100303915
:1095100009291AD80C00A74223DD591C09D063463B
:10952000824206D302D10499A14202DB012378438F
:1095300020182C780135E9E72E00BCE72B2C01D050
:109540001E00C7E7B51C7478FAE7210041391929D4
:1095500001D8373CDFE721006139192901D8573C90
:10956000D9E75A1C08D1059A23331360029B03984C
:10957000002B09D107B0F0BD002E00D04042029A66
:10958000002AF7D0002B01D06B1E0193029B019A99
:109590001A60EFE73024002FAAD10827A8E7302C63
:1095A0009ED00A27A4E7C046FFFFFF7F37B5130010
:1095B000064A05001068046A002C00D1044C0A0019
:1095C00000942900FFF770FF3EBDC04660000020F8
:1095D000C4000020F8B505000E001400002804D0D7
:1095E0008369002B01D100F0C1F9224B9C422DD19F
:1095F0006C68A369A360A3891B0731D52369002B7D
:109600002ED023682269F7B2981A6369F6B28342B2
:1096100005DC2100280000F03BF9002826D1A368D2
:109620000130013BA36023685A1C22601F706369EC
:10963000834204D0A389DB071AD50A2E18D1210052
:10964000280000F025F9002812D00FE00A4B9C42B8
:1096500001D1AC68CDE7094B9C42CAD1EC68C8E7A0
:109660002100280000F00CF80028CAD0012676421C
:109670003000F8BDFCB500001CB60000DCB50000F1
:10968000364B70B51D6806000C00002D05D0AB6987
:10969000002B02D1280000F069F9314B9C420FD118
:1096A0006C680C23E25E93B219072DD4D90611D44D
:1096B00009230120336037331343A381404270BD37
:1096C000284B9C4201D1AC68EBE7274B9C42E8D188
:1096D000EC68E6E75B0713D5616B002908D023002F
:1096E0004433994202D03000FFF79AFA00236363B3
:1096F0002422A3899343A381002363602369236009
:109700000823A2891343A3812369002B0BD1A02135
:109710008022A389890092000B40934203D021004C
:10972000300000F0E1F90123A289134011D0002399
:10973000A36063695B42A361002023698342BED1B9
:109740000C23E25E1306BAD540231343A3810138EC
:10975000B5E7920700D46369A360EDE760000020DD
:10976000FCB500001CB60000DCB5000010B50620FA
:1097700000F0E0FB012000F01DFD0000F7B58A8934
:1097800005000C00130760D44B68002B04DC0B6C45
:10979000002B01DC0020FEBDE76A002FFAD0002379
:1097A0002E682B6080235B01216A1A4034D0606DE3
:1097B000A3895B0706D56368C01A636B002B01D0D1
:1097C000236CC01A0200216A00232800E76AB84708
:1097D000A189431C06D12B681D2B30D82B4ADA40B7
:1097E000D3072CD50023636023692360CB0405D500
:1097F000431C02D12B68002B00D16065616B2E6089
:109800000029C7D023004433994202D02800FFF733
:1098100007FA00206063BEE701232800B847431C15
:10982000C6D12B68002BC3D01D2B01D0162B01D124
:109830002E60AFE74023A2891343A381ABE7402307
:109840000B430120A3814042A5E70F69002FA1D05F
:109850000B680F60DB1B01930023920700D14B695B
:10986000A360019B002B00DC94E7019B3A00216A76
:109870002800A66AB047002803DC4023A2891343CE
:10988000DFE7019B3F181B1A0193EAE70100402024
:109890000B6970B505000C00002B01D1002070BDD4
:1098A000002804D08369002B01D100F05FF80B4B36
:1098B0009C4209D16C680C22A35E002BEED02100E3
:1098C0002800FFF75BFFEAE7054B9C4201D1AC683B
:1098D000F1E7044B9C42EED1EC68ECE7FCB50000EC
:1098E0001CB60000DCB50000002310B504000360C6
:1098F0004360836081814366C28103614361836108
:10990000190008225C30FFF782F9054B246263627C
:10991000044BA362044BE362044B236310BDC046B7
:10992000759F00009D9F0000D59F000001A00000D2
:1099300010B5024900F08CF810BDC04691980000A7
:1099400070B568254A1E55430E0029007431FFF793
:10995000B1F9041E08D000212A00016046600C30D5
:10996000A0606832FFF753F9200070BD836913B51A
:109970000400002B28D18364C3640365134B144A8D
:109980001B6882620193984201D101238361200008
:1099900000F020F86060200000F01CF8A0602000BB
:1099A00000F018F80022E06004216068FFF79CFFD7
:1099B00001220921A068FFF797FF02221221E06827
:1099C000FFF792FF0123A36113BDC046A4B50000B9
:1099D00031990000F8B51C4B07001E68B369002BD5
:1099E00002D13000FFF7C2FF4836B4687368013B0C
:1099F00004D53368002B07D03668F6E70C22A55E45
:109A0000002D0DD06834F2E704213800FFF798FFED
:109A100030600028F0D10C2304003B602000F8BD2A
:109A200020000A4B656625606560A560E3602561DE
:109A30006561A561082229005C30FFF7E8F86563DD
:109A4000A563A564E564E9E7A4B500000100FFFF94
:109A5000F7B504000700002601914834002C01D11D
:109A60003000FEBD6368A5680093009B013B009336
:109A700001D52468F2E7AB89012B08D90E22AB5E31
:109A8000013304D029003800019B9847064368350C
:109A9000EBE7EC300068704770B50E001D000E2338
:109AA000C95E96B01400002907DA00232B60B38941
:109AB0001B0611D48023DB000FE06A4600F0D8FAC1
:109AC0000028F2DBF022019B12021340054A9B188A
:109AD0005A4253412B60EDE740230020236016B02B
:109AE00070BDC04600E0FFFFF7B502268B89050078
:109AF0000C00334206D02300473323602361012347
:109B00006361F7BD01AB6A46FFF7C6FF0099070026
:109B10002800FFF7CFF8002808D10C22A35E9A0591
:109B2000EFD4032293431E43A681E4E70F4BAB62BD
:109B30008023A28920601343A381009B206163617D
:109B4000019B002B0DD00E23E15E280000F0A2FA4D
:109B5000002806D00322A38993431A00012313434C
:109B6000A381A0893843A081CBE7C046319900008A
:109B700082B0002900D101A9101E06D0002B06D00A
:109B800013780B601078431E984102B07047022092
:109B90004042FAE7C9B28218904201D100207047D2
:109BA00003788B42FBD00130F6E710B5884202D92A
:109BB0008B18984203D3002307E08B5C8354013A4F
:109BC000FBD210BDCC5CC45401339A42FAD1F8E701
:109BD00070477047F8B507000D001600002905D141
:109BE0001100FFF767F804002000F8BD002A03D138
:109BF000FFF716F83400F7E700F072FA2C00B042D5
:109C0000F2D231003800FFF755F8041EECD02900DD
:109C10003200FEF7F3FF29003800FFF701F8E3E711
:109C2000F0B58E6885B007000C00039201939E4248
:109C30003CD890238A89DB001A4234D00325096975
:109C400023685B1A0293636902985D43EB0F5D1909
:109C5000019B6D1001331B18AB4200D91D00530549
:109C600032D529003800FFF725F8061E09D10C234C
:109C70003B6040230120A28940421343A38105B0E9
:109C8000F0BD029A2169FEF7B9FFA389144A1A4070
:109C900080231343A381029B2661F6182660656129
:109CA000019EED1AA560019B9E4200D9019E3200E3
:109CB00003992068FFF779FFA36800209B1BA3602E
:109CC00023689E192660DAE72A003800FFF782FF32
:109CD000061EE0D121693800FEF7A2FFC7E7C046A3
:109CE0007FFBFFFFF0B59FB0029005938B890F00BB
:109CF00016001B0611D50B69002B0ED14021FEF773
:109D0000D9FF38603861002805D10C23029A013848
:109D100013601FB0F0BD40237B61002306AC63617C
:109D2000203363761033A37635002B78002B01D0D7
:109D3000252B46D1AB1B04930CD03200390002987E
:109D4000FFF76EFF431C00D1AEE06269049B9446AE
:109D5000634463612B78002B00D1A5E0012200232E
:109D60005242626002A9543252186E1C2360E360B2
:109D7000A3601370A365317805225448FFF70AFFEA
:109D8000751C00281FD12268D30604D5532302A9CD
:109D90005B1820211970130704D5532302A95B18FF
:109DA0002B21197033782A2B16D0350000210A2078
:109DB000E3682A786E1C303A092A4ED9002918D057
:109DC00010E00135B1E7414B2268C01A01238340FE
:109DD000134323602E00CEE7059B191D1B680591D8
:109DE000002B01DB099304E05B42E3600223134391
:109DF00023602B782E2B0AD16B782A2B35D1059B2B
:109E000002351A1D1B680592002B2BDB0793304E81
:109E1000297803223000FFF7BDFE002806D040233A
:109E2000801B834022680135134323602978062272
:109E300028486E1C2176FFF7ADFE00283CD0264B4B
:109E4000002B25D10722059B073393430833059345
:109E50006369039A9B18636166E7434301219B187A
:109E60003500A6E701235B42D0E700230A201A0051
:109E70000135636029786E1C3039092903D9002B1C
:109E8000C5D00792C3E74243012352183500F1E7DA
:109E900005AB00933A00114B2100029800E000BF8F
:109EA0000390039B0133D3D1BB890B985B0600D48D
:109EB0002FE7012040422CE705AB00933A00074B07
:109EC00021000298FFF700F9EAE7C046A8B50000B4
:109ED000AEB50000B2B5000000000000219C0000FB
:109EE00070B504000D001F2904D91623036001205A
:109EF000404270BD436C002B04D08A009B181A6846
:109F0000002A08D1200000F031F82A0001002000CA
:109F100000F01AF8EDE70020012AEAD0511C03D125
:109F2000162301302360E4E7002428001C609047DA
:109F30002000DEE710B5034B01001868FFF7D0FFE3
:109F400010BDC04660000020002370B5064C05001F
:109F500008001100236000F0FFF8431C03D12368C0
:109F6000002B00D02B6070BDBC25002010B500F088
:109F7000E3F810BD70B50C000E25495F00F0B8F88D
:109F8000002803DB636D1B18636570BDA389024A5B
:109F90001340A381F9E7C046FFEFFFFFF8B51F00AC
:109FA0008B8905000C001600DB0505D50E23C95E64
:109FB0000022022300F080F8A389054A28001340FC
:109FC000A38132000E23E15E3B0000F02BF8F8BDC8
:109FD000FFEFFFFF70B50C000E25495F00F06CF835
:109FE000A389421C03D1054A1340A38170BD80227E
:109FF00052011343A3816065F8E7C046FFEFFFFFFE
:10A0000010B50E23C95E00F021F810BD0B1E04D060
:10A01000FF2A04D98A2303608B3B180070470A701B
:10A020000123FAE770B50500080011000022064C74
:10A0300022601A0000F0B6F8431C03D12368002BFD
:10A0400000D02B6070BDC046BC250020002370B539
:10A05000064C05000800236000F05EF8431C03D1A5
:10A060002368002B00D02B6070BDC046BC250020AB
:10A07000002370B5064C050008001100236000F0B5
:10A0800053F8431C03D12368002B00D02B6070BD14
:10A09000BC250020002370B5064C05000800236095
:10A0A00000F052F8431C03D12368002B00D02B6032
:10A0B00070BDC046BC25002070B505000800110029
:10A0C0000022064C22601A0000F04EF8431C03D117
:10A0D0002368002B00D02B6070BDC046BC2500203B
:10A0E0000B1F1B68181F002B01DA0B58C018704794
:10A0F00070B50500080011000022064C22601A000D
:10A1000000F03AF8431C03D12368002B00D02B60E9
:10A1100070BDC046BC25002058220120014B4042A2
:10A120001A607047BC25002058220120014B404294
:10A130001A607047BC25002058220120014B404284
:10A140001A607047BC2500205822024B00201A607C
:10A150007047C046BC25002058220120014B4042D8
:10A160001A607047BC25002058220120014B404254
:10A170001A607047BC25002058220120014B404244
:10A180001A607047BC250020044A1368002B00D1D8
:10A19000034B1818106018007047C0460C120020BE
:10A1A000C025002058220120014B40421A60704710
:10A1B000BC250020FEE7C046F8B5C046F8BC08BC88
:10A1C0009E467047F8B5C046F8BC08BC9E4670472E
:10A1D00054050000640500007E050000FC05000039
:10A1E000340600006A060000A2060000C80600004F
:10A1F00004070000460700009C070000E00700007D
:10A200004C08000094080000BA080000F2080000A2
:10A21000380900005E0900008C090000BE0900003A
:10A22000F60900007A0A0000460B0000BC0B000093
:10A23000280C0000700C0000900C0000B20C000014
:10A240008C0D0000D20D00005405000054050000E4
:10A25000540500004A0E0000B20E0000340F00004A
:10A260007A0F0000C20F000040100000BE10000076
:10A27000061100004C11000082110000C8110000FE
:10A280000E12000056120000AA120000081300006F
:10A2900046130000B0130000E61300002E14000067
:10A2A00076140000BE140000F814000040150000F1
:10A2B00088150000540500005405000054050000F6
:10A2C000F0150000261600005C160000881600003D
:10A2D000BE160000F41600005405000054050000EE
:10A2E00054050000540500002A1700006C170000F8
:10A2F0005405000054050000B217000002180000C9
:10A300002818000054050000540500005405000002
:10A310005618000086180000B6180000EC1800005F
:10A32000161900004C190000761900009E19000053
:10A33000C6190000F6190000261A0000501A000085
:10A340007A1A0000AA1A0000EC1A00005405000056
:10A350005405000054050000540500005405000099
:10A360001C1B0000481B0000741B0000A01B000009
:10A37000CC1B0000021C0000381C00006E1C0000FA
:10A38000A41C0000D01C0000FC1C0000321D0000BA
:10A390005405000054050000540500005405000059
:10A3A0005405000054050000540500005405000049
:10A3B0005405000054050000540500005405000039
:10A3C00054050000540500005E1D00008A1D0000B9
:10A3D00066616C73650074727565006C69737420D6
:10A3E0006F66202564206974656D73006F626A650D
:10A3F0006374206F6620636C6173733A2025640078
:10A40000537461636B20756E646572666C6F770060
:10A41000070000000300000059A40000651E0000B2
:10A4200061A40000691E00006AA40000611E000013
:10A4300073A400006D1E0000150000000100000064
:10A4400002000000040000000500000006000000FB
:10A4500043616C6C696F706500686173546F6E6501
:10A4600000706C6179546F6E65006861735365723A
:10A47000766F00736574536572766F00496E7375FD
:10A480006666696369656E74206D656D6F727920AB
:10A49000666F72204D6963726F426C6F636B7320DD
:10A4A0006F626A656374206865617000496E7375D8
:10A4B0006666696369656E74206D656D6F7279207B
:10A4C000666F72204D6963726F426C6F636B7320AD
:10A4D000737461636B000D0A564D2050616E6963A1
:10A4E0003A2025730D0A006D69736300FCA4000017
:10A4F0007523000005A500002D2300006865785431
:10A500006F496E740073696E0000000058A500006A
:10A51000E123000060A50000E52300006AA500001B
:10A520000324000073A500000D2400007EA5000098
:10A53000172400008AA50000212400009BA500002C
:10A540002B240000B1A50000EF230000CAA50000E5
:10A55000F92300006E6574006861735769466900ED
:10A560007374617274576946690073746F705769C8
:10A5700046690077696669537461747573006D7913
:10A58000495041646472657373007468696E67440E
:10A5900065736372697074696F6E00636C65617274
:10A5A0005468696E674465736372697074696F6E2D
:10A5B00000617070656E64546F5468696E674465BD
:10A5C000736372697074696F6E00617070656E6438
:10A5D000546F5468696E6750726F70657274790059
:10A5E0000D0E0F04050C0B0A0607080904050C0BD9
:10A5F0000A06070809000000000008080800080A09
:10A600004A4000000A5FEA5FEA0ED92ED36E193283
:10A610004489330C924C924D0808000000048808CD
:10A6200008040804848488000A448A4000048EC414
:10A6300080000000048800000EC000000000080038
:10A6400001224488100C9252524C048C84848E1C3B
:10A65000824C901E1EC244924C06CA525FE21FF00A
:10A660001EC13E02448ED12E1FE24488100ED12E10
:10A67000D12E0ED12EC488000800080000048004EA
:10A68000880244880482000EC00EC00804824488F8
:10A690000ED126C0040ED135B36C0C925ED2521C82
:10A6A000925C925C0ED010100E1C9252525C1ED026
:10A6B0001C901E1ED01C90100ED013712E12525ED4
:10A6C000D2521C8808081C1FE242524C12549814A3
:10A6D00092101010101E113B75B131113935B37144
:10A6E0000C9252524C1C925C90100C92524C861C54
:10A6F000925C92510ED00C825C1FE48484841252CE
:10A7000052524C1131312A44113135BB7112524C25
:10A710009252112A4484841EC488101E0EC8080850
:10A720000E10080482410EC242424E048A400000CC
:10A73000000000001F0804800000000ED2524F10DD
:10A74000101C925C000ED0100E02424ED24E0C92A3
:10A750005C900E06C81C88080ED24EC24C10101C0D
:10A7600092520800080808024002424C1014981443
:10A77000920808080806001B75B131001C9252525D
:10A78000000C92524C001C925C90000ED24EC20003
:10A790000ED010100006C8049808080EC807001252
:10A7A00052524F0011312A4400113135BB00124C76
:10A7B0008C9200112A4498001EC4881E06C48C8402
:10A7C00086080808080818080C881800000C836020
:10A7D0000000000001000000020000000300000073
:10A7E0000400000005000000060000000700000053
:10A7F00008000000090000000A0000000B00000033
:10A800000C0000000D0000000E0000000F00000012
:10A8100010000000120000001400000016000000EC
:10A82000180000001A0000001C0000001E000000BC
:10A830002000000023000000260000002900000086
:10A840002C0000002F000000320000003600000045
:10A850003A0000003E0000004200000046000000F8
:10A860004B00000050000000550000005A0000009E
:10A8700061000000680000006F000000760000002A
:10A880007D000000840000008B00000092000000AA
:10A8900099000000A0000000A7000000AE0000002A
:10A8A000B5000000BC000000C3000000CA000000AA
:10A8B000D1000000D8000000DF000000E60000002A
:10A8C000ED000000F4000000FB000000FF000000AD
:10A8D00020A90000512400002BA90000212900001C
:10A8E00035A900003126000042A9000051260000D1
:10A8F00049A90000A126000052A90000F12600008D
:10A900005EA900004D2900006FA900006528000025
:10A910007CA9000031280000646973706C617900C3
:10A920006C696768744C6576656C006D6244697328
:10A93000706C6179006D62446973706C61794F6607
:10A9400066006D62506C6F74006D62556E706C6F56
:10A9500074006D62447261775368617065006D6266
:10A960005368617065466F724C6574746572006EF1
:10A97000656F506978656C53656E64006E656F50E5
:10A980006978656C53657450696E004E6F7420650C
:10A990006E6F75676820726F6F6D206576656E20CB
:10A9A000616674657220636F6D70616374696F6E48
:10A9B00000436F6D70616374656420466C617368F9
:10A9C00020636F64652073746F72650A256420626A
:10A9D000797465732075736564202825642525299D
:10A9E000206F6620256400426164207265636F7287
:10A9F0006420666F756E6420647572696E67206985
:10AA00006E697469616C697A6174696F6E0025643E
:10AA10002025642025642028256420776F726473C4
:10AA200029002564207265636F7264732C2025648D
:10AA300020776F7264732C206D61784944202564FF
:10AA40002C20636F6D70616374696F6E206379632E
:10AA50006C657320256400526573746F72656420A1
:10AA60002564207363726970747300537461727427
:10AA7000656400726164696F000000000AAB000049
:10AA80005933000017AB0000C535000027AB0000AC
:10AA90006935000035AB00004537000040AB0000D1
:10AAA0007133000050AB0000E533000064AB0000E0
:10AAB0008133000073AB0000253900007FAB00003C
:10AAC000A538000088AB00004938000093AB0000B7
:10AAD000913700009EAB0000CD370000A7AB00000F
:10AAE00001380000B0AB0000953300006E756D6258
:10AAF0006572006E6F6E65006F74686572007061DC
:10AB0000697200737472696E670064697361626C64
:10AB100065526164696F006D657373616765526545
:10AB2000636569766564007061636B657452656323
:10AB300065697665007061636B657453656E64006A
:10AB40007265636569766564496E746567657200F0
:10AB500072656365697665644D6573736167655495
:10AB600079706500726563656976656453747269AE
:10AB70006E670073656E64496E7465676572007315
:10AB8000656E64506169720073656E6453747269B6
:10AB90006E67007365744368616E6E656C00736503
:10ABA0007447726F757000736574506F77657200CB
:10ABB0007369676E616C537472656E6774680000C8
:10ABC00000000000963007772C610EEEBA5109990B
:10ABD00019C46D078FF46A7035A563E9A395649E67
:10ABE0003288DB0EA4B8DC791EE9D5E088D9D2978B
:10ABF0002B4CB609BD7CB17E072DB8E7911DBF90E7
:10AC00006410B71DF220B06A4871B9F3DE41BE840A
:10AC10007DD4DA1AEBE4DD6D51B5D4F4C785D38366
:10AC200056986C13C0A86B647AF962FDECC9658A0A
:10AC30004F5C0114D96C0663633D0FFAF50D088D66
:10AC4000C8206E3B5E10694CE44160D5727167A20A
:10AC5000D1E4033C47D4044BFD850DD26BB50AA566
:10AC6000FAA8B5356C98B242D6C9BBDB40F9BCAC8A
:10AC7000E36CD832755CDF45CF0DD6DC593DD1ABE6
:10AC8000AC30D9263A00DE518051D7C81661D0BF0A
:10AC9000B5F4B42123C4B3569995BACF0FA5BDB866
:10ACA0009EB802280888055FB2D90CC624E90BB10A
:10ACB000877C6F2F114C6858AB1D61C13D2D66B666
:10ACC0009041DC760671DB01BC20D2982A10D5EFCA
:10ACD0008985B1711FB5B606A5E4BF9F33D4B8E826
:10ACE000A2C9077834F9000F8EA8099618980EE1CA
:10ACF000BB0D6A7F2D3D6D08976C6491015C63E626
:10AD0000F4516B6B62616C1CD83065854E0062F249
:10AD1000ED95066C7BA5011BC1F4088257C40FF5A5
:10AD2000C6D9B06550E9B712EAB8BE8B7C88B9FCC9
:10AD3000DF1DDD62492DDA15F37CD38C654CD4FB25
:10AD40005861B24DCE51B53A7400BCA3E230BBD4C9
:10AD500041A5DF4AD795D83D6DC4D1A4FBF4D6D325
:10AD60006AE96943FCD96E34468867ADD0B860DAC9
:10AD7000732D0444E51D03335F4C0AAAC97C0DDD25
:10AD80003C710550AA41022710100BBE86200CC949
:10AD900025B56857B3856F2009D466B99FE461CEA5
:10ADA0000EF9DE5E98C9D9292298D0B0B4A8D7C7C9
:10ADB000173DB359810DB42E3B5CBDB7AD6CBAC025
:10ADC0002083B8EDB6B3BF9A0CE2B6039AD2B17441
:10ADD0003947D5EAAF77D29D1526DB048316DC739D
:10ADE000120B63E3843B64943E6A6D0DA85A6A7A41
:10ADF0000BCF0EE49DFF099327AE000AB19E077D9D
:10AE000044930FF0D2A3088768F2011EFEC20669C0
:10AE10005D5762F7CB67658071366C19E7066B6E1C
:10AE2000761BD4FEE02BD3895A7ADA10CC4ADD6740
:10AE30006FDFB9F9F9EFBE8E43BEB717D58EB0609C
:10AE4000E8A3D6D67E93D1A1C4C2D83852F2DF4F40
:10AE5000F167BBD16757BCA6DD06B53F4B36B2489C
:10AE6000DA2B0DD84C1B0AAFF64A0336607A044140
:10AE7000C3EF60DF55DF67A8EF8E6E3179BE69469C
:10AE80008CB361CB1A8366BCA0D26F2536E26852C0
:10AE900095770CCC03470BBBB91602222F2605551C
:10AEA000BE3BBAC5280BBDB2925AB42B046AB35C40
:10AEB000A7FFD7C231CFD0B58B9ED92C1DAEDE5B9C
:10AEC000B0C2649B26F263EC9CA36A750A936D0280
:10AED000A906099C3F360EEB8567077213570005DC
:10AEE000824ABF95147AB8E2AE2BB17B381BB60C00
:10AEF0009B8ED2920DBED5E5B7EFDC7C21DFDB0B5C
:10AF0000D4D2D38642E2D4F1F8B3DD686E83DA1F7F
:10AF1000CD16BE815B26B9F6E177B06F7747B718DB
:10AF2000E65A0888706A0FFFCA3B06665C0B01117F
:10AF3000FF9E658F69AE62F8D3FF6B6145CF6C16DB
:10AF400078E20AA0EED20DD75483044EC2B303397F
:10AF5000612667A7F71660D04D476949DB776E3EDB
:10AF60004A6AD1AEDC5AD6D9660BDF40F03BD837FF
:10AF700053AEBCA9C59EBBDE7FCFB247E9FFB5305B
:10AF80001CF2BDBD8AC2BACA3093B353A6A3B4247F
:10AF90000536D0BA9306D7CD2957DE54BF67D923DB
:10AFA0002E7A66B3B84A61C4021B685D942B6F2A7F
:10AFB00037BE0BB4A18E0CC31BDF055A8DEF022DDB
:10AFC000416C6C207461736B732073746F70706567
:10AFD00064007630363900202573202573004D65D6
:10AFE0006D6F727920636C6561726564004E6F20CD
:10AFF00066726565207461736B20656E7472696535
:10B000007300000044B00000FD49000050B0000093
:10B01000194A000056B00000494A00005CB0000028
:10B02000CB49000062B00000894700006CB000000E
:10B03000794A000074B00000B548000073656E7373
:10B040006F72730074656D706572617475726500FE
:10B0500074696C74580074696C74590074696C7408
:10B060005A00746F75636852656164006932635297
:10B07000656164006932635772697465000000009D
:10B08000F4B00000FD4A000002B10000014B0000D6
:10B090000BB100000D4B000015B10000114B00007A
:10B0A0001EB10000154B000023B10000194B000039
:10B0B00028B100001D4B000034B10000214B0000FE
:10B0C0003BB10000254B000044B10000294B0000BB
:10B0D00049B100002D4B000054B10000314B00007D
:10B0E0005EB10000054B000068B10000094B000094
:10B0F00074667400656E61626C65446973706C613E
:10B100007900676574576964746800676574486599
:10B110006967687400736574506978656C006C6960
:10B120006E65007265637400726F756E646564525B
:10B1300065637400636972636C6500747269616E43
:10B14000676C65007465787400746674546F756319
:10B1500068656400746674546F756368580074663B
:10B1600074546F7563685900746674546F756368BE
:10B1700050726573737572650057656C636F6D65AA
:10B1800020746F204D6963726F426C6F636B732123
:10B1900000705F73706920213D204E554C4C002F8C
:10B1A000686F6D652F62726F6D61676F73612F2EAF
:10B1B000706C6174666F726D696F2F7061636B6123
:10B1C0006765732F6672616D65776F726B2D617243
:10B1D0006475696E6F6E6F726469636E7266352F27
:10B1E0006C69627261726965732F5350492F5350B5
:10B1F000492E63707000535049436C6173733A3A3F
:10B20000535049436C617373284E52465F53504903
:10B210005F547970652A2C2075696E74385F742CC0
:10B220002075696E74385F742C2075696E74385F90
:10B23000742900000000000000000000394D0000EB
:10B24000F54C00001B4D0000254D00002F4D000067
:10B25000194D000000000000010000000200000085
:10B2600016000000040000000500000006000000B9
:10B270000700000008000000090000000A000000AC
:10B280000B0000000C0000000D0000000E0000008C
:10B290000F0000001A0000001B0000001400000056
:10B2A0001300000011000000030000001000000067
:10B2B0001C0000001D0000001E0000001200000025
:10B2C0001500000017000000180000001900000021
:10B2D0000000000000000000E951000019590000C2
:10B2E000695200007D52000073520000E5510000D9
:10B2F000D95100008952000005520000D5510000CC
:10B30000000000000000304300000000000030C3D7
:10B31000FB21F93FFB2109407CD91240FB21194058
:10B320007A6A1F407CD92240BBFD2540FB21294081
:10B330003A462C407A6A2F405C4731407CD93240F3
:10B340009C6B3440BBFD3540DB8F3740FB213940DF
:10B350001BB43A403A463C405AD83D407A6A3F4096
:10B360004C7E40405C4741406C1042407CD942409A
:10B370008CA243409C6B4440AC344540BBFD4540EF
:10B38000CBC64640DB8F4740EB584840FB21494045
:10B3900083F9A200444E6E00FC291500D157270006
:10B3A000DD34F50062DBC0003C999500419043001C
:10B3B0006351FE00BBDEAB00B761C5003A6E2400EE
:10B3C000D24D42004906E00009EA2E001C92D1004D
:10B3D000EB1DFE0029B11C00E83EA700F5358200F8
:10B3E00044BB2E009CE98400B4267000417E5F00BF
:10B3F000D6913900538339009CF439008B5F840067
:10B4000028F9BD00F81F3B00DEFF97000F980500EC
:10B41000112FEF000A5A8B006D1F6D00CF7E360092
:10B4200009CB2700464FB7009E663F002DEA5F001C
:10B43000BA277500E5EBC7003D7BF100F73907003F
:10B4400092528A00FB6BEA001FB15F00085D8D001D
:10B45000300356007BFC4600F0AB6B0020BCCF00F5
:10B4600036F49A00E3A91D005E619100081BE60016
:10B4700085996500A0145F008D40680080D8FF00AA
:10B4800027734D0006063100CA561500C9A873007F
:10B490007BE260006B8CC00000000040FB21F93FA4
:10B4A000000000002D44743E000000809846F83CE7
:10B4B0000000006051CC783B00000080831BF03915
:10B4C0000000004020257A38000000802282E33608
:10B4D000000000001DF369350200000003000000B9
:10B4E00004000000060000008873000032730000B2
:10B4F00032730000607400002E7300002E73000091
:10B5000056740000607400002E7300005674000032
:10B510002E73000060740000647400006474000006
:10B52000647400006C740000887F00008A7E000054
:10B530008A7E0000A8810000847E0000847E0000D6
:10B5400090810000A8810000847E000090810000AE
:10B55000847E0000A88100009E8100009E81000082
:10B560009E810000AC8100002C2066756E637469BA
:10B570006F6E3A2000617373657274696F6E20227A
:10B58000257322206661696C65643A2066696C6582
:10B5900020222573222C206C696E6520256425737A
:10B5A00025730A0064000020232D302B2000686CD6
:10B5B0004C006566674546470030313233343536D6
:10B5C000373839414243444546003031323334350F
:10B5D0003637383961626364656600000000000038
:10B5E000000000000000000000000000000000005B
:10B5F000000000000000000000000000000000004B
:10B60000000000000000000000000000000000003A
:10B61000000000000000000000000000000000002A
:10B62000000000000000000000000000000000001A
:10B630000000000000000000000000004300504F28
:10B64000534958002E0000202020202020202020B8
:10B6500028282828282020202020202020202020C2
:10B6600020202020202020881010101010101010F2
:10B670001010101010101004040404040404040436
:10B6800004101010101010104141414141410101BE
:10B69000010101010101010101010101010101019A
:10B6A00001011010101010104242424242420202A8
:10B6B000020202020202020202020202020202026A
:10B6C0000202101010102000000000000000000016
:10B6D000000000000000000000000000000000006A
:10B6E000000000000000000000000000000000005A
:10B6F000000000000000000000000000000000004A
:10B700000000000000000000000000000000000039
:10B710000000000000000000000000000000000029
:10B720000000000000000000000000000000000019
:10B730000000000000000000000000000000000009
:0CB74000000000000000000000000000FD
:08B74C00BC49FF7F0100000071
:10B75400FFFFFFFF400600001800000019FCFFFF78
:10B76400FFFFFFFF0200000003000000FFFFFFFFD8
:10B7740000000000010000000000020001000000C1
:10B78400FFFFFFFF000000000200000000000400B3
:10B7940002000000FFFFFFFF0000000003000000A4
:10B7A40000000800030000000A0000000800000078
:10B7B4006400002000000000FCB500001CB600007E
:10B7C400DCB50000000000000000000000000000E4
:10B7D4000000000000000000000000000000000065
:10B7E4000000000000000000000000000000000055
:10B7F4000000000000000000000000000000000045
:10B804000000000000000000000000000000000034
:10B8140000000000430000000000000000000000E1
:10B824000000000000000000000000000000000014
:10B8340000000000430000000000000000000000C1
:10B8440000000000000000000000000000000000F4
:10B8540000000000430000000000000000000000A1
:10B8640000000000000000000000000000000000D4
:10B874000000000043000000000000000000000081
:10B8840000000000000000000000000000000000B4
:10B894000000000043000000000000000000000061
:10B8A4000000000000000000000000000000000094
:10B8B4000000000043000000000000000000000041
:10B8C4000000000000000000000000000000000074
:10B8D4000000000043000000000000000000000021
:10B8E4000000000000000000000000000000000054
:10B8F400000000000DA00000719B0000000000008B
:10B9040046B6000044B60000E6A40000E6A4000029
:10B91400E6A40000E6A40000E6A40000E6A40000FB
:10B92400E6A40000E6A40000E6A40000FFFFFFFF79
:10B93400FFFFFFFFFFFFFFFFFFFF00000100415378
:10B94400434949000000000000000000000000001E
:10B95400000000000000000000000000000041534F
:10B9640043494900000000000000000000000000FE
:10B9740000000000000000000000000000000000C3
:10B98400E9000000C54C00000D50000035550000D2
:04B99400C1000000EE
:04000003000050A900
:00000001FF
